:040800003FEF5DF079
:08080800160FF66E080EF72230
:100810000900F55012006A1A578DA42265E508B048
:1008200039093AED42A6BCC164BCB71A33B554A924
:10083000852EACF51E97CEA799A850D93186C31A3C
:100840000B9F7353E360E957AE77D572DE32DCDD80
:1008500023C2C51AF7885E85143B3B19F612CEF108
:100860006899E9C8668F031B78158294158C9AEFF6
:100870003F1F1B7B690E31518CF8041BEE9388F1EE
:1008800062D9E25B7F44F14871C8A61F3518091B85
:100890001670528B917D2FD99F0B981063EB8D8929
:1008A00069DF211BF8390D2ED9AF79DEEFCE6A7AD8
:1008B0001F500A795C092C1B8618EACAB8C0D90FE8
:1008C000328540EE15374DE9C5D2341B1BD2F4A456
:1008D000B5CE5F16E1D99AF5EA88D6C3F3FE491B77
:1008E0007427CB7B52A31E631AE8FA1F754FBFCF44
:1008F000CE58501B0670A6204B4E4CB32577DA9786
:10090000D78FDBBB3C3F5B1B3443FB35CE1BE5C2C3
:10091000705956384410A2B3024A5F1BD6FEDC82DF
:10092000D8268850379D9D2C312ECA40BFC99A1BAE
:10093000CCB0620ED622432C213D4DCDA9F5001C32
:1009400072F2A21B7112FB2B6610C7A9585E4CDD18
:10095000F2CF2E863B1CCE1BC5345E34822EC508DA
:10096000161D01285FA6B4A5641BD51B23923AB4BB
:10097000F658A8E207C5A4B9D634CDB5A4B0E91B92
:1009800084045E8DC887621DAFE82A9D950461606E
:100990003FE5FF1B79069F1B883A96F8A32BD77279
:1009A00056E292E0B098151CEF319D6C95B1C40DE4
:1009B000BF75A020884BFEEE5E9D231C1325F871A9
:1009C000D36BDC4A6B9759CFAEF97C1128CA2B1C2C
:1009D0008A1D30B62D14B4141666B00445BDF1213D
:1009E00021942D1CD521EAF2641055813E2B31450E
:1009F000560A04CC8BA49A1C0955695A9ED20752F8
:100A00000ADD54BADB72FD1C763BBC1C6812F5A3F0
:100A100045D79AB3896E76F7B871CF90D6D3BF1CFD
:100A2000EDCB436EEBEAD067D79D55163289F9318D
:100A3000EB17D11C0A599445CB34EF854D0799E546
:100A40004568BE460104DB1CD595849A10AE9FAD67
:100A5000BF73D94A0F7225F1A7D0F01CB45EB778E6
:100A600034E8A9B41A2A5244050B8CB1449AF11CFB
:100A7000A5787CF539E4738BA9267B5F817A93296D
:100A8000DEA0F61C30EF33F1DAF7FBDD11835C6694
:100A9000B76ED6ED205B251DED8F590ABEF4F640EA
:100AA00074C39B54D26A3DD69F50361DD03A5D1F09
:100AB000F8EF8E4D2962BEDE1A9F84DE4185401D0F
:100AC000703475F0C4873BFE9202CF76B5B6F78DD1
:100AD0009D6D4E1D6F7EE9D396745A4E337CC626AB
:100AE0006F9AEA24A79D541D246B35C61A0B4398B0
:100AF000DAC8AB5B4CDBFEB647D5601DCE3C7D9DB6
:100B000076628888DC9C1720061532342DE7731D29
:100B1000A062BDDA8C28BAC26061029C92CEA4C9E0
:100B2000B6F0DD1DC197D4FD80095FCD0DE808E466
:100B3000A48CE6EA75D4FA1D54DC7358EF69CD90A5
:100B4000739340BC2F7B387B6C58031E54616DBE81
:100B50006C068B8024D3008DCA2FE6CD8440511EB5
:100B60007E0CB7205152FF2C9A34D70C3E8561433E
:100B700029487E1EAADE6926BCBCC679FB518B982B
:100B8000B8DED8C416159A1EE981301C8A6C989775
:100B9000152EE3DDF22A9C3559D5AD1E1C8C7ACF7B
:100BA000DCCC268FECF391E89EEAE0F0B632F11E41
:100BB000B0B26BA771D0BD3D8F937CC4CF6FDE0800
:100BC000236DF31E168561342C192E777DC9B7A1CC
:100BD0006EE3DB609706261FFB8BDEA55FF7A96E31
:100BE00048A751A64F923259F4764D1F7C9A75D082
:100BF00060F87F4D80CB4468C864870A71116C1F10
:100C0000B43AA2157F302D3F5E6923AE14E338B0AD
:100C100002FC841F11DAE07A8DB31E55C1E71C7DFA
:100C20003CF3FDA542478F1FC51827E1DFD337925C
:100C300029BC29509FCCB24553AF911F85D0DC9E73
:100C400021EDE32FD9B9B4BA9B6A2831D20AA01F8B
:100C5000E10CEDB4E279A1317C7462B100E7249635
:100C6000F6E3AC1FC53CC67D78A6A1749E4513D1A2
:100C7000807CCB29F838B61F55C17BD709C3810FBB
:100C80004847AB7F21BBB9CA21B1C01F2BDA5FEC4B
:100C9000BD2F298DF1CD790ABCBAA2C63D1DCA1F50
:100CA000C296BB8AFD147DB00A76ECC49D208E02EC
:100CB000C1B8E91F42C5518F1A94FBA357DCD6F87F
:100CC0008FEAF48D772A0420AA28717D1FD58E8B98
:100CD000C95AF8FBD0045B829CBD0A2063EB63A277
:100CE00016D9D320CC39A8B29389EEB334B91720E2
:100CF000506302F50199887836723EC0D3201EDF1A
:100D00001FDC4F20496836A7BCCE512979562C6E7E
:100D1000E867F6FDF2657020B19278831BEB69619C
:100D2000A0B667A91571CEE141387A2035F2884224
:100D30008612A55A9FB59FE0A946AFD26E2E7D20A0
:100D40007F6C71A422459D99EFD3C017FFC17994A0
:100D500022C3852039F8FA043F6608ABE8268321D0
:100D6000398D2991A068B520919B0DD0CAD36ABC5A
:100D70003AF69D34C5F5A1595EB0C820947A3292F6
:100D80005E2C53AF39550B67C5BDA9B3F7D1CF2042
:100D9000D70C35F55BCC72EAAF7D881B1C3838C6A2
:100DA0006F27082144228C685C689DAA8B95E961B5
:100DB000CE8BFBCA156B4421560083E6E9E932A8C5
:100DC00086D2948256E85BA4F257452193E77F3F91
:100DD000FEED3F6D659FB5BB752DB1111F344921E7
:100DE000A1B86D200741DE74E2FAD5705C8DA5E6EE
:100DF00011785F21F4B14E88ACFF73F5BB81A41765
:100E000002A2AEE39A0A602134AA7A40D51C14FDEE
:100E10005826A39B7BEED57295F889217F49354CE6
:100E2000B52FE5B4A6EB621150C1B2FE9319C221F1
:100E300061E23263C1D18F6013CCFBF77CECD457F5
:100E4000F9BECD21A607D29111913DE96E3858A582
:100E50009D71C664F516D0218A4A1BA7A4DF826B58
:100E600004F3CB9ECB16B0799E91DE212996D8FF54
:100E700064A4FBB9E07CC13EA90BD44F9EA8EC2131
:100E8000035F2909EDBE39230090733C2C1C5844A4
:100E9000C97EF2218585C9DCA0B1C40A6FCDF405F5
:100EA0009CC69A9DF45AFC217E3FFBA0B89170E24B
:100EB00066DC6B333351E13E372F12221AF4C194B2
:100EC0002440873B50208FF1F980444D996E452294
:100ED0004A0A9A95AA4945BB28D2244A06532A11A0
:100EE0005C63822279CFE10EEC4DDD660ABCC03135
:100EF0005C3ABF090707882212BFB5323077D23576
:100F000060F721C02B34BD5A9BE993226B36C4860F
:100F10006D6DCB805C4CBD47F460AF3670CFAE22B8
:100F2000951083DA463E40ECF352EA9424A743EA54
:100F30002862B222F209BAB45C487C2C001E70C947
:100F40000ADA9D4DC2E6B322E04FF13F3604ED1EB2
:100F50004FD2965EE164E4C03E22BF221BCD2970D1
:100F6000A8CBA1649B30F9D5DE68DE40D65ED722DF
:100F7000CDFFC7D144E102BCCA7E753FF5D2163F12
:100F800001AED92264813AF740BA7619010E23C422
:100F900016FF62EB8E71E122AADBE73AE68B3ACECE
:100FA00027A1D38BFB5D49E81D181623875B578863
:100FB000A112A41E9E496AE4BCB567D533811A23E9
:100FC000B0214770900ACA1F3D4878371B8180ECDA
:100FD000B85A6C23D90C296121CCBFAE26C33D88F9
:100FE0003A7F390BDF8E812378EA1A1257B0D3E5A6
:100FF000E3CD540A8E1A6E92323B9723700249BD9C
:10100000134441CEA11C6E7B7CEBAA30168CAA2324
:10101000242DF65A9B7BA3604FBD4920361B3768B1
:1010200081FBB6236EB13CFEF61DD97AAC3D620160
:10103000FB5BFF140F9CBB23B7A199CCB489EAEFEB
:10104000D0659DD51E4F380E5BA4C2232D14C6F962
:101050001D50C790146D5775E69843D9E78E042448
:101060001B7D7F909C878AF6640949F0F64D207AB3
:10107000CBF108245FCF1A6813111D4FFD8974410D
:1010800032DB887D62C70C24D63C4217185F53FBC5
:101090007726DBB713AD88EB983A2C241F332BDF70
:1010A00022BD4D5FCD19495C154DFFEE50DE402449
:1010B0004EEA5CEEEA518F594E783901BD5AF33B46
:1010C00098AF42240BFFB6BB97DBDE5B06213C17D3
:1010D00009B3D869FC0251243DCCA7647D4675DB79
:1010E000561837FAE1FA905776847724DD49624B37
:1010F0001C77435A617F218F34D604EEF38E8C2403
:1011000075EB3D0BE7818156ECAD57797D565A1A48
:10111000D75493240111081EBC26ABC4C779E1251E
:10112000611337CA5D75A8247706BB7BCBAFB5CFFB
:101130007CD8691AE8C652CCE0DCC22454C90070DD
:101140009B11913EBB678ABFD85B3E757AC6D72498
:1011500088104C756B16FD94FDB9F45F18B7C6EB9B
:101160006F14D92412F0E514AF2C6BE8C4258898CD
:10117000B36AFFACB84B01255A3A533D5BA5AC4C62
:10118000BAF6BA60036F799D50C40825C31D28754F
:10119000FC70F47468120DE2B7A7BE17694E3125D2
:1011A000B71E22E326B04D84B711CC5B311A52949E
:1011B00056C95325F3FC43AD7B08BF8E64C41B3F67
:1011C0005700E7626B505425E80549ADDD24E40182
:1011D0000BB3CE3E142AB2D9BE6F6525A00C5910B0
:1011E0002F760C0C5F133C0E1AB9676B33A466257F
:1011F0009A7293A551E869D60836B9705B21570AEF
:101200009EAB672531C987C60236582057E011408A
:101210006D7CFEC07BFD80251EDF6C88244813702A
:10122000EAEC5A979F1C123217E28525A3E253CFAE
:101230006C52FE491AD12F00EA5F8F252B2CA02576
:10124000733C255C40BF1B835D76D9D44E9F4B0E0B
:101250008AE8AE25F9AF7FFD3D8477FF9012DC9FD1
:101260005C63A49112E6AF2558B31B7645259A71AD
:1012700092CCDCFE0D2A058663C0CB255A63F1E7CC
:10128000F7647E411D28D64B4BAD8B9CA8DDCF2546
:10129000C4D5A7AA2F4307626007F5B0DF8FB5F763
:1012A000F4A2DE25F4D8678B73921FC283CF0D277B
:1012B0000A418DCDE00B1A26EFBE595055F1F6B21A
:1012C000C38513583A3F047E47A269260A6952B281
:1012D000621E853EC52E57AA889503A2D0F67C26AD
:1012E000D2F5AEDE892B0264E1317FA3DE0AB6DEE1
:1012F00002158E2660B63DA0D19065BFA51DB4E055
:10130000BD06CF5C91FCEB266BF79DD3410922CA49
:101310007B91BB62400C637D10D20E27B9A0D370C5
:10132000698F1C62E745964D22C296FB3C651027EB
:10133000D098DC3553250B332FB326FE8FDAD42615
:10134000B56C5F27EB2EF34CCE8AD5AD69F6A28043
:10135000D05F2D728C468227C6769140D3BF80DA4B
:101360007C5221FB270719EE97C0A0270C1EA970FD
:101370003BCFBEA4A8C956E3409730032A86A227D4
:10138000C5444D3EFCFA69207EB0F8EC419B05FE59
:10139000BF2CBD27DFD647D155FB8C37B5376F1D26
:1013A000BA93AC969508C82703C287E1AD02DB76F5
:1013B00072BFC731A363283816CED627262E09C799
:1013C0002354BAA49870F83BD4BD64AF4A9DD72784
:1013D000CE1B5850DAE5C178EEE0DD52299B7A7BCE
:1013E000B175DE273604F82279D3D2DC0AC7522839
:1013F0007E5014B50CADF9271CE2B7509E3AC31AC3
:10140000C740B2A3E30903916B0E552855F5D242AC
:10141000BA1F8E74BE5527FC49FBFB29137D6F282C
:101420000D1E88F34DF6AB61E98B53730D719CC8AB
:10143000B74AB128DA7C35C442F7476D6EAD5055D6
:10144000E1B594119DBFCE28C245DF60E980D3FD90
:101450004A03A1EC563609EE0D40D0288194ECA841
:101460009A1AD46215AAA38BC326F6C79EAADF28B0
:10147000278C7CFC7B1EC1B0E65B5EB30BC2646F45
:101480004BF3F7288B171660B1469C830739E52785
:10149000CC6BC3F22E4647296296360EB96DD3F651
:1014A000ED9D21A15A654A2FF3F75929F9FD7A409C
:1014B000D52E893B3F7AB8579FF22C8DF3CD9329D7
:1014C00057B4AE571354AC6FD9A314D665D408845F
:1014D000B5EF9D2992EF66270CF3F325632AF28B73
:1014E000C370D3C82D4EAB29157E66897EFAE455AC
:1014F000F21009F0528D0A6EF774CE291E3D00D00D
:10150000F91340A8650BC9BBA4E0E8002FDD0E2A43
:10151000889630B618B3FE4A26310BE70717A0C0ED
:1015200068E5132AC8970D187FDEBDCA2989F48E95
:10153000AB45E01FD671192A0A6BA20178571A33FE
:10154000F75B0C8349D74BA4C66F2E2A18D71A70A5
:10155000E80F0F409D699302E1EC6341AAD14E2A46
:10156000C66E93E39B901D9F62F98BEBD8121F48C8
:101570000D32522A65860FC23EEBB4A1EBAB1E7D45
:10158000B55A18E7AB818A2A8372751E599D2E576A
:1015900099EA16F48656D72091D9BA2A02336B4DB0
:1015A0000C014E944F8E12E413B79B8C06A2CF2AE7
:1015B00040776BC38038D9FCE99DCC738BE332EF65
:1015C00017AF0D2B2608BFD58E64C167F29AC9A943
:1015D000770AAB87A01D222B93DE5592634849BF43
:1015E00050CBF7021186A4BFFECE4A2B416CF9F511
:1015F000EC77ADAA4972650AE22D824C75F16A2B2F
:1016000002EFE48420CCB38E7E4E3B1C7593B05A1F
:10161000BF4B752B4375040E4FAC169334819F96C8
:10162000BF4C271AF0F47B2BFB019B0EE846DD8AAA
:10163000E4887E8B821C9B294F638A2B99C23CC510
:101640003C59222496D3179C029569696A2C8D2BEC
:10165000E6615B8E128CF64150C224D51B330C75AB
:1016600093E7C32BEA67F036FB7A4B835F8CCC9D04
:1016700094746F9FDEFEE22B9C7804A526380D71D2
:101680004E19F813A5CFE1216F3FF52BFEF86DCA77
:1016900050B0C6381BE045814F484B4E076AF82BC7
:1016A000FFC7F35BCE31451CE2BB4FB0BEC46AC27C
:1016B000ED9D1D2CE9F675CD4EF5C6E941528EFF24
:1016C0007F8A81BA24CF282CF8B79AEEB45E57519E
:1016D00065EC52AF98E5CDE7DDD4362CF1720FDA28
:1016E000301C349A82C5E880E794C9B64E4A3C2C37
:1016F000FC2B3E71E24DCC7DE11B390C073135AD41
:101700009FDF4C2CBBF004F3D165EF4B352FB36753
:101710000676BF65FF334F2CD1DD30588188BEA6D9
:101720000B99B5A339331619B12F5A2CE8536CB164
:1017300057DAA8EC75045282EA6652B4473F652C2A
:1017400053240E2C0722CEF1769DC8EFB10B1C530B
:10175000BA296A2C13D9E9A7EB71582E7ACFD5D0C4
:10176000C6FE503B2D2B6F2CFB5D32C6510010ADD9
:10177000743988961D3C6A25FF29722CFE9810BD8D
:10178000DD229A808D78513BF8B8F57B56F2882C93
:10179000500256BD4121AE54148EEADFD35814D006
:1017A00062F08C2C21FA04566BC65FA2A5786E906D
:1017B000E68474B0691D902C44785830E46AC014F3
:1017C000F77E4E59C1572495AD399E2CD432213B1A
:1017D0007D66FD050DE55F52A34E97FBAD16DB2C34
:1017E00053826A77FB8D4A5D801725D18C70A137B3
:1017F0005F23042D65B0890917591FAB7DD6058776
:1018000060C5ECF40CAE182D160FC73874A59DE416
:101810003268361050793F89B016542DD23567930F
:101820000071BAD7C1323CFCF10FFF84FDE1852D78
:10183000A5786C2FE564CE292A2A473FC2B94D31DD
:101840002382882D958CE3EA509EE803DE5E528F5A
:101850002EA9A663E45A972DDEE51F207E2E1444A0
:10186000656FCEBCF0815660A688D72DD5FD8B5F05
:10187000DF89B10DCDA0DACAC29FAD217DE3EB2D8A
:10188000291F9D881904E0B412BED53C09C0D1922D
:101890007275202E54B8106A8DDEF30E729E0457B6
:1018A000B12EC6A95A2F242E0405D3422CC5B82820
:1018B000CAA0E7C29AC86E3D876C542EEBC80A9D39
:1018C000B568FCB1DC70A92A1B4FB2434C96632E5D
:1018D00030742F3191E4982A5928230467805CFDE5
:1018E00080EC742EEF7CEE1059F9439F325B694E09
:1018F000B41B939BEF3FA52EF3928B134D638E95F4
:101900009BD8B8FF60C5B60D2670AB2EA95A00A6AD
:101910005028F2F04FAD73F4412D33444606AE2EFD
:101920004610898EC5C37E766F94D1B34C5524651D
:101930008058B02E6302B2975B9A2C4133EAC4EC14
:101940003525BAFD3140C12ECB97C395ABE98B57F6
:101950006735FCA1C4A66F4E4952D32E405F19359E
:101960002A12BDE1242831FB3D0BAD95C5ABFE2EFF
:10197000F5C140B5672AFDC9CC921DD6C33D20C92B
:1019800027D6032F2E149E258F683B49BBEF1CBF23
:1019900011ABF1EC0A0A122FA66209B1705C5AEE83
:1019A000DF18472243CE496B75D13F2FE3B6CC8E6B
:1019B000897C8AD4FF1436412623F5603975602F5F
:1019C0003AEF592F9B9C4EC29E1A1B4B849684B8AB
:1019D000BDC7842F36B0F765D5F8879ABC256872E5
:1019E0000856395F2CBB8D2F6D29815FDA5F6FBE82
:1019F0002CD754A3605BAB426AFE902FDB1203CC62
:101A0000F423B3016DBBB8426E76033F7C39A12F3E
:101A1000BAE8436AE00A29002390ED118956EDA93E
:101A20003FE5FA2FEC8E66D46E4EEAF1CFE6FA86E9
:101A3000CAA976A12051FC2FF14CD13152175ABAC4
:101A4000CBAC382A389A96C7AC00FE2FC00CD4FC19
:101A50004CF22526E894D94D8FBE114E4AFA053036
:101A6000444F492AB0AFBD5C59F7B547098A54A223
:101A7000B95F4430F71C0F66A87F5D0B5BB5E3A42C
:101A8000BD59DB2F679F6F3045D38CD017C6961199
:101A9000A2ADE256EB19482F0B108030DE537C14B8
:101AA0009E7CB7C1D646E5E273726D5851E2843030
:101AB000DF1D74F78B1CF6336576D6E27D841E92AB
:101AC0005A389D3078D23F8B4A957BAD14F2C91CB1
:101AD000E1A41388A45AA0309D4CE5F006BB8B5EB0
:101AE000AD8B9E6405E838C59054B4302827CEDB12
:101AF000B6E7D16D4B9BC361162852E4F66CD0302B
:101B000029348232F81B30DFFB2B435B9CF151A957
:101B10002FB4D7304EAD288CE33EA1D8293AD87BDC
:101B2000191AECCBBE6EF030B5DF151EA0A4844EA2
:101B300091B62C6D4FFB4E9FBDD4FB30C7E4653E84
:101B40006354800F3DA812ADDA7BFAD287221B3195
:101B500074C3014492DF6B88CE69C13D910498162D
:101B600007C41C31FDFC2A363EF8DD82A3DEC247E5
:101B7000ACCBE9EC0CC42131746CA9E13A538BCFA6
:101B8000CD12FA9BAA650C914EBD37311921AF8950
:101B900069DE4CB40572FA7EE4F3134E08A361319A
:101BA00099BEA729E94C08F33C497EFA7B50A49FD3
:101BB000E10E6B314F4D3A23BE8DFC60A7DF027FF3
:101BC000DD0C0178F119A7313C50A7BD21C0D97AAD
:101BD00022D77071BF44D6305743D131DDA2FF0CFC
:101BE0004A29BF7F407898D3E76734BB3146133228
:101BF0009C7114CFA98DC2A19EE3D43E3B499FA105
:101C00005DEF17320E6868C207A8F073CE58C3F4B0
:101C1000BB5918D2537E4D32015245403F97A527FC
:101C20001284D90A6E6378C150A362328441DBE921
:101C3000F8B67B0B9786B5DDD127090F78846A3219
:101C4000506B398BBBA7CEFDD9B69E8C85A9EC70A5
:101C500069148932A3B278B54B5BCAB3283A142E03
:101C6000FB24A3136EE69532BAFB68DCE3F806307A
:101C7000667059A28B53ED897563D3324828D5B36A
:101C800044D29DE18F20C0864B1C97898A0CEC3290
:101C900004EA18BAEA830CDEB094747234254675EF
:101CA00077D1EF3273DAAE61C11B2CB2FF98FFE837
:101CB000C079B9DBF6CA0833103CBB16F6F51C1820
:101CC0000B48BA9CBB979F961D2A0A333D81E77348
:101CD000C5701AA67E8267C7A56D52BD45321933FD
:101CE0007BB2ADE278116B836EC23FC46C994961DF
:101CF00086E725333D4DE2CCE1620837C15CF7A0B1
:101D0000CCA4B3D279C3383387579E67DB40EDB696
:101D10002B0726D1F1226C69E38E6F33170AB86F57
:101D2000F05387A945B98A867DF9C8BC26D39D336F
:101D3000C6E210205129647BB6B12D749D03D013E7
:101D400091C7D03332C683C220304B24A12F6DC639
:101D50000BB6459CADB8E133EA6C530BFD0A86E146
:101D60008753215D7BBE8DAB7E4EF63361A558A6B1
:101D70009E7A1E3B1F3EB496400382059D4AFA336D
:101D80005631ED333A64D9B0ECF2B0129348614C5D
:101D900030C85C349E01B4C38BC6D7B7403EA44262
:101DA000B1CCA74FBECBBC343492616A7C286FDCC7
:101DB0007240DF7D13CCAFB8CE4CE6344DEF19C383
:101DC000FA8427B60F97A1F121C5DAA1672E313524
:101DD0008F253712291237865AF8B628C875186C1D
:101DE000AE694C35DDC2B25E9A1059A0E7909742B9
:101DF0009CFBF88202D65135AA7597EC608F45E1BD
:101E0000C1D33730D8108B90A7DB5335C20F0411E4
:101E10009ADB12EEF044D1995C5999483BE5B43510
:101E20000614E99597F95582EFE3196F706719DE8B
:101E3000B707C635FA79E41E14FF221D0A556DF561
:101E4000797DA0F514B0DC35D0C2F62F49823AB7BF
:101E5000EAE02C049802B229B88AEC35AA56A7A960
:101E60004A1D54D8A8477B64FC84C9B4EB6E033682
:101E70000D023781A04B9382B8F05F0DF5BC7BDE7D
:101E8000A2260B366D21ECA3AD95D468479DEA22BE
:101E9000842349A196952C36F43A4333A76813CC92
:101EA0003DC13DF8C942DEBEC09F2D36EFF1C642AE
:101EB000CE98CD184F393202A56B96DAA9EA3D3695
:101EC00092FAE4269919B531695FC19177F629F242
:101ED000776F4836DBD7AFDC94C4046EA7F1126687
:101EE000161EEA9D2B2E6336E17AF2591A7CD5ED47
:101EF00025E15DC2628A8A10BFC1943624C32D4F8A
:101F0000D6A2935A8535B653ABF851DB147FB2365F
:101F100047541EFA74E5DD96D970A0654A838CDFBC
:101F2000D851B83664D6391669263C864CA862EF7B
:101F3000F7BBF5A0F31DC036E0094A5D438D13835E
:101F40002DAFE8D4F43292BCC7C0C636C7218B0887
:101F500057165EF95DC2D6147E5C2C87D069CB36ED
:101F6000373B54AEE0F3CD87E1FA06BB3703D97BAC
:101F70009E05CC36BE35CD8AD3B453512420675943
:101F8000766236B5B8FBCF369595D29C649A3956B1
:101F9000F2845337C6BB3F9AA3BAD936A364109CC8
:101FA0000CADE1093C67B6398CC59A22D9DDE23621
:101FB0005DDD0BC2E29DDB61F5E35935BA08E4C58E
:101FC000CE660537AC3FE0CE81B91C6247BDF4A0B8
:101FD0008E5CCA8D4F67153749F8DC2C9CE3189747
:101FE000757300E5688F8B3A8FE92D3705FE894DB3
:101FF00090B721ED9EFCCC78756BDBA64EC13237D5
:10200000E6AE2DAF82E968D26C1E4218F87C2E0332
:102010009E4837377B44889BA6827E66E3CC33B5E7
:1020200050959143B07441375DE2280F972CE9DA5F
:10203000A0F8EB1F5B9523DD56AE56371C3E2B7187
:1020400035B3E1DC05D4DE4A2189578D8F1467371B
:10205000097A31A65983A041873B269CE3840FAEC1
:1020600094DCA637BD2EBCACB4CADAA7B181AB04F0
:102070004A4362D39AF1B737E863319120C94BDC08
:10208000DB770F3302D16C077008D337397F06B581
:10209000B921BD87CF1857936997B894EC3DED37B8
:1020A00022966F8E55B73B084EE15A6706DB430711
:1020B000511903382EE61F9CB1473FC09FF0697D40
:1020C000B8B10B3E4A29053880B43BCCD3F94ADE7F
:1020D000AEC5DA6D5408F6F28D221C384C67E570F7
:1020E0007E64E8093D6DDFD4215D538E807A3138FE
:1020F00043D98350ACDCACD6FC01883134D4DA420D
:1021000096BF6438D256081355774CF2B2AA5F1FB7
:102110003C7E5DB7DA8B67389D9335745D700BD765
:10212000EE840841EC31A9E8AAC886386B1EA8E8FD
:1021300046756D2BE9F0EEA9870AFF3CB831AD3842
:102140004D4DC26D44634341F6336CB1F2D0677EAE
:102150000AC7BA38EC18C9E00C732C79A690D327BB
:10216000CA0A20BF0751EB38319C0F93A4841AE4AC
:10217000563FAAB95ACF9BC93454F738B6ECAAF3E4
:10218000043031E24222278081B3FDF9837706399A
:10219000B8D55A1CB68D038AB99DABBF1947EF7EDF
:1021A000EE7A1839F0C1097E4DCC5C3EAF119C47E8
:1021B0001BC76082CC2141394FCBEAA7D337CE4F22
:1021C000527CD9504D93C31AEB2E95395A58F88A40
:1021D000B56A8E719830E0875F9F48729D23B7394A
:1021E000CA35DE5F32EF7304628D3E015BAA3C1C90
:1021F000D1E3C239863EA61E006ACE9CFEFF75F270
:10220000AAF0B2EBC7BEEC390AC042B5EF57A6CF71
:102210002197333E81913AC96984043A04069CF4BB
:1022200021240C614B34D5F0B64F02ADB27E193A81
:10223000256A522B1174BB7B1FCF4C260B8953048C
:10224000C370433AE583E7E70223F48D14C744F8EB
:1022500029FC3AA6040D4A3A214B9C890FF91AF43D
:10226000408AC5DA11C7EAF04C157D3AF8B64B281A
:10227000046019CCEC519D9A5AA423056885873ACD
:102280005192919F40C68E1C402813FB5A69EF055E
:1022900063868C3AFF67CEE951C29DF30ABDA06206
:1022A000790641A53F5C993AC8EF8EB4FFDE9805E8
:1022B000151AF2B30D7D01E73EF09D3AD7BF5BA73B
:1022C000A33B300C045E04298C72FB79AD26A63A40
:1022D000A92668B5785E25FA305C08554A8F394DD5
:1022E0002060BB3A55F64E92C4ED3619A0C82AA418
:1022F0001802DBA65849C13A7D98B9CADA19DD90AF
:1023000041F75AE315EB474409CFCA3A5E9A789CE5
:10231000496378D06676911E324FABD68B50EF3A38
:1023200018B2D1310CA8111FCE80AB1527CB5B3B67
:10233000C78C093B6A3B2CF619BB2E151F2EB473B4
:102340007C7833FB000B243BD074BF64B27BC1109C
:102350004C1BB29530147E6F946B4F3BC8E6EBBDBF
:10236000BDA9ABB975BE07029E2B3F0BEC836A3B40
:102370002056AE153F8CC8142D0E4EAA1784064465
:102380005084DC3B3FF1B400ED64E8A37A025E6662
:10239000B9A0320F9B27ED3B7701A1B166C2482659
:1023A00034AE845B88171A0714EA103C288D352256
:1023B000D49B0513327F81D139214C1E032E123C50
:1023C00063667A380B6F58FAEBC9D57BF65A98508A
:1023D000AD2C503C3D6B54426C889B33853E3B6238
:1023E000D120570FCD9F743C39E6891EE0B8A43840
:1023F0000576C7E556663EB052CFA03CB86BA95BE8
:10240000347B3EF5ECADE0FC3864E5725D77C33CAF
:1024100076CFC563158227B715A571669E6C9F950B
:102420005193E03C70982049CB3E12CFA5634F6793
:1024300078E99E00E4BAE23CADAB9247F91AEDBBF5
:10244000EBB539FB905AD41DF309F43C8BFF410CDA
:102450004EBE831AC39169E13AA34A2D1DF8F93C97
:1024600052B3DAFFBF0611951B45CE819E6AC22189
:10247000D086293DB380CC3FC5D95FA7351BA5B811
:10248000C2933DAA7F12373D3D17149E185DDFEBC6
:1024900013753150D0C5C9A3D9C74D3D03F54208C6
:1024A000BA13B098AE92B43E84610966CF8B533DA7
:1024B00072857A43F245790880DBE0D5B12390D369
:1024C00082F0973DFBB6D67F73A6C9F70B73423EE9
:1024D00027645FF5F8BE993DE16FD374B120B27CFB
:1024E000E29DCF4E3BC0C5A974CBC23D565AD1FA2E
:1024F000988151DF260FDA0F62383FBEE675D43D72
:10250000063382934CC88723E89035EAE78F934BD4
:10251000D366E93D32F3AD696BDCDA6F66DE3E7F90
:1025200059FEC91D987EEF3D0908996DC84F867701
:102530009FB5CD629B2D78C72869FE3DB83C297CAC
:1025400040D6AC0FCDB25BEC902F1C711CC25A3E32
:10255000D2DD819CE10AE9A607CCF699E940FCF3BB
:10256000529E643E2A900EA3A467F74583F16B4BFD
:10257000784CE53BFF766F3EA67A18B9F36BA5E879
:102580007D59EDD0B1567955B41C743E76211C743A
:10259000C469CBB2DA83F407DC8A6229E0367A3E7A
:1025A0003F34D7824E656955A9A9C1980D6E06C4FE
:1025B00081D4803E2A211D24C84FD5DB388C42F8B7
:1025C000102C25CDA609933EB682858BB581940E3D
:1025D000826E6D87F1C15FEBF96DB33EB8769237CD
:1025E000F036565D15148949870975ED7BF0D53EA7
:1025F000D8E2B2BB3343020A1B79390190E3FC8570
:102600007414EE3E71EAB4433E4097D603BAD71E27
:1026100008B7A7D562CDFF3EDE09A1D9B1E68C0D82
:102620005204125AA222B7725ED3073FBF95DBBA9B
:10263000E7EE44340C6A17F002F795876962153F9C
:10264000323B43F430F0C017A8079AF9CB41FAAEF9
:1026500075DA1D3F30C2B7A2ADC65EE1AA5FE9726E
:10266000D32484D8DCC8633F7B6ECF649FF18D6335
:10267000361B4EEA035F39DFCE4E663F6D1DB22D2D
:102680005C8E5D81030CF550CF4FBF58D05C723F1C
:10269000FDDBD2F80BC639E8F595527D6E91D5EC8D
:1026A000B3EB7D3F641B7C3EDEDB0D2FE5C47D0A72
:1026B0005E648AE6D4DD863F00E8414BEEB535190D
:1026C0008C8483B2826BF6B18B0B893F54C9DEBF19
:1026D000187543242226830A9C87474BA9A1A03F53
:1026E0005349C6D7263CFB14904735900947442EE2
:1026F0009CB8AD3F4C2EA4AD2B2C5968AAEE474593
:102700001BC1E9B2C8AAD13F862592CF06D430B802
:10271000C02F9E7A87343262A6BDDA3F85143DDA37
:10272000F55EC5E135D485C009DFEB2F263EE73FD6
:102730004F71B8DC0DB46235026591F7A7E86C60A3
:1027400002EBE83F6AB8ECD822398D0CA9238B291B
:102750002C52F285C8C11240968D91CC389CE85419
:102760002EA169B0B18C114F6E994240DBE5BC815E
:10277000BE528516D44E54DD1EB137490AB64B40C1
:10278000B2AA64A71DCBD797D5DE313BC3F9B79565
:102790008DB7624088116BC3122B8E518B7A9032A9
:1027A0009C18885D05367E40769414EDD5C4C59698
:1027B000679096C9C3BB6F4386BB864044AF4AF857
:1027C0002CDD2ED191326D89A39A23AB3F9C8A4098
:1027D0003C785DCEF1295A2427E9D98647740596BD
:1027E00075B68F407349ADDF81489BD48D9761D911
:1027F0005B14AE7AAEF899407D24CB0A47053AD7F0
:10280000CB5B53973BCEAFA87789E040D65293D7A6
:102810007B90080C37F47C5C52AAE9E9CF01E540D3
:10282000211B6BC72D9570931DD9782820629EB906
:102830001807EF403AA915B11876FCBF2C5399D46C
:1028400019026CB1A7A3F140BAD9963F68D38C9610
:1028500021FA48186A7A4B5F659F40411CEECC987C
:10286000989B52F844DF85583C63C25BB2A77C4119
:1028700009E244C0BBC735EB8963BEF98E580D4EE3
:10288000774BB041D746E311680DDA2D51222F93D3
:1028900085F862503F40B8416F62016F885E42BE6A
:1028A000C32572BDF06C3E668A39DD417FEDC8A458
:1028B000C4B0EA04E50E2EE99664BABBBA16154216
:1028C000102219BCCC76ABB450C923DC73A69FF19F
:1028D000ABF63C427A0E499225397B66E57F0DC105
:1028E000109176A6A4F24342D545F522157EBA4A48
:1028F000B50C567915A616FA905A7842521E98B71A
:10290000A59305923BF0A9EF1C8C087F22E17E4243
:10291000DF6C1AD999C822276A4BA14E2A3FD67B71
:10292000E1BD864255343B49E0757A2164A5D01259
:1029300065ACE46E9931904252D2CD3459705F4506
:1029400077A28BF4369ADE00477C994204F5B1B346
:1029500019593F458F41AAA183CE7832236AA942F3
:10296000E3BC33E9B02518B5221EDF09FED9945126
:10297000D813B04267C174206FAADE1DC5A590CBE5
:102980008A6F04CE134DE0428AAF156A6FE8FF8E5E
:10299000F6CA21BF63F0EABA1C2DF7420DC706B292
:1029A0000D07B5666019FDD43BBFB256CE1528435E
:1029B00027D4DFD1032D9F3EB1F1A8DC9B43F3DD8B
:1029C00022D13143123E0FC6221DFA8221BF8A4C0A
:1029D000BBA84CC342275A436A8426D6A2421F7A18
:1029E0001B5C7FF84F8510EE3C7D7543C64799DA36
:1029F000C171E536A9E32B8CC9114BA13A55A0430F
:102A0000DAAA139FE3A81C6CAB3309F1246EDD80B6
:102A10002390C0431330B3A7E41CA8E7B6B3832ABE
:102A200063463F8811FFC343E353B750F3676287A0
:102A300053372EFA70B09D4A545DEA43CE69EFF9E0
:102A4000DAA071E6BB33EEA6C71916D538CF2444F9
:102A5000104F7A51A11F5471A4F26082BC16C8A015
:102A6000EA663D448BE4594DFC43ED332559D04D86
:102A700058E08C5E1A854D4490F3E11287B1DADBA1
:102A8000BB28D79674937BF8B2B26244622359D3C1
:102A90008476707ADF28D6786FC1EEFE3CC19F4401
:102AA000F18AA4FDA2A3CB90723F21189D7985BD28
:102AB000A9D1CB4442FF45842A5F4622D535BAB31B
:102AC00023EF2B32E8A8CC443C11CDE38CF0CE941C
:102AD0000F3CCCF7C274D01778BAD1441427142213
:102AE0003029CF3E3C6BB3DD9251C317F19BF544C7
:102AF000A9AD79E207527CCF231AF8BA401D4F28BE
:102B00009D020345AECBD6858E4207E9DDACD803E6
:102B1000F91C0000FCFF09455652DF2EBEE4698710
:102B2000405C0F024ADE237C9B320C452EF0CAD655
:102B30001B731084044BA6F64B8F03C80C432B4524
:102B400001D0348D0D723AB8A8513EB815E81FE295
:102B5000DBEC344504B2FA2EE3D11BF7CF901C65B1
:102B6000C38B582EFF2678455E1BFAF73CFF0BDA25
:102B7000C980DA15DA3B23D72FD27F451062AAC667
:102B80006519CF58F6642584EFB0CF0A12758445D5
:102B90002BE5B26DE4482FDA7DD520B8A8A07A23C2
:102BA000C8E0A8459AA1135928D4E30376DF189FFB
:102BB00084575CF74C33B8459F6FF7F1CDC6D79E6D
:102BC000150D2D1D8E978FDD4887F64562FD42F36A
:102BD0003F5FD8CB4A1764823FB88468F075FA45E6
:102BE000EAB994A011EFB5D90C938C1A3C6AF2B8EB
:102BF0004B630046A296F711782451A8CC10ACFD87
:102C00006B85591681770A46878ECF97BA15D0AE55
:102C1000FD433DFC7D8350241A771B46BB6037BEC5
:102C20006670CE8DAE0D3FB1ADA4F267EF0F2846B2
:102C3000CC23F3CC0823C0DD0A2CBBB5DD38722CC5
:102C4000DD2139462306AF3AC3EC39B32B55860E46
:102C5000B170783F29E24C466B4CBCA9E2769713E1
:102C60008686EF97ED18096B90CC794634C16BF2EC
:102C7000C3127767ADD054FD21EFCA7A45857A46F5
:102C8000529F9356D9E05C7BC7FB334CD119699EA8
:102C90000C587D4612BC788F78E9C5185B8C158876
:102CA0007E070FB435029346B72DD2077606F01A89
:102CB00064B3BA71C1C3B52AFA8FD746A2D52537F6
:102CC000FA71455F6857046F7EDD96CDB484DE46A9
:102CD0006499971E28E6824AEBCAC849703657198C
:102CE000D0B9FA46389C4499EFA45944C63E0E8E9A
:102CF000F7990DA8197A0647DD813FF8FFCC801AB5
:102D00000BEC85F425444017CFC11E475B84FAB411
:102D1000C104D4891F3B0A2C1649DD0106922D47B8
:102D2000EA3221C1C922B99C6D8A2206450D3A1AA0
:102D30001E31374728B29DB1D8ED81E29977A67050
:102D4000ECBF408D80CF3A4771BAA950CD5E4306A3
:102D5000537A0B0927A2B07EA445A547130A35FD77
:102D600004FFB99FB5D7C740733824905C43C4476C
:102D700077612FF62C706F25CCC6868CB423DF9537
:102D8000E6DEF747250F4D33C0BED3589C46E9FE1B
:102D90009635A46B81831248636974609838F7A1F3
:102DA000595588D9C97D9BD8FCDE1448CC716E6F0B
:102DB0007417ABEAB656151AD16FF01DCD1E1A481E
:102DC00027BDF37B4CE044DC299926DC4F928B71C4
:102DD0006F8D2648E5C8839F4D58F82F9C16FE61DD
:102DE00014414772C8B92B483F8FE4E8C309CE3B72
:102DF0007A78FF1B06F72F5C38933A48C0945D4001
:102E0000C52F10D6FB38A01BA459BA71F2F23C486A
:102E10002050F59922915BEFFDA824E989EC876F9A
:102E200012CF4248EAAF6E2FF4318918254C5FA7C4
:102E3000A3D2556069D76F48BEA4C309099350094E
:102E400095D93F25C2A47D769F5E7648B2DC048783
:102E500017EE01CC6B6849CA4D1E709FBCF28748C3
:102E60005B2C9BBDC0CF936B1A5B74C71100BDE890
:102E7000F4AC94480198A7424AF99B853DF74D5E12
:102E800090152C9382F6A94839BFD03FA10011328A
:102E90001C219167425438B17FC3BA4873B2D847F6
:102EA00047ACCB1BEBE295A2241D5531CA59CB4848
:102EB0000F0DA50EE7FD42DDA6B7B236311737BAC2
:102EC0002EE8ED48E151397B66894656A5CBAE61C7
:102ED00059D6F222763E08494E3C078017759E234C
:102EE000C79A79120066E3D2DE720B4941FE4B5A53
:102EF0002EDF5F9152D12BC44864FF71ACDA3549A3
:102F0000ABB4FF3051D3378FC6263936C74CC58A8C
:102F1000A5926249A6BF9D95AD264A468EB7FD1281
:102F2000AABAE61378C0BB49DF5E284034766F53F7
:102F30003AFA5443A8929B38CE7AC549D34ABA612B
:102F40007EB03890FE2567AB9DEA923E1FE1F449C2
:102F500036FB582BF34D9442656D301142F21594B7
:102F600047CF0E4A3D11602476A394955815D2C2DE
:102F7000A544A971A224174A409A91C901B837778C
:102F80000DB52DE573C0766364B0194A7704B614A5
:102F9000B3A50ACA9579C11BC077115380C63D4AB3
:102FA00018BD0E1449673305723B0F4194FE3F3B39
:102FB000C21C434A81CD13EC3289BA5F742D71BEB5
:102FC000D8F1709F4661464AE35340D094F8FFD849
:102FD0001F7F3954BB46A61D13064C4A0CE62CA194
:102FE0004BF9CEE9AB9A3FDB80AD260986256E4AC8
:102FF000134DD5C90F855968768881EA912305E478
:103000005C80864AE959DADBD28DBC44804022BD1F
:103010002E4199E0B97F9E4A25D8ACE2FFD4D86012
:10302000B4F04EE07CB5740A48CDDC4A1F92C13B37
:10303000C9DDEF23FB0721D30E89C6BCC1BC174BEA
:1030400056E668199BA14D2F880996780DAB9CB266
:10305000A7BC694B5E2DF300E1E5771B65D6A3C4E1
:10306000116546092C22904B2587FF05949E442428
:10307000868EF1F82C1D645C77F3A04BD3661D3D62
:10308000ADF31EF7EA678195555EF7AEA840A14BF8
:10309000766F0F3F4ADC729F4FF4252603C9C6A9FD
:1030A000D484A64B1CEF24E2823FADC6D42C771605
:1030B00024A6FCDF1ED4CB4BAF7FE8571015AE9E85
:1030C00021DFF3A6B473B1FC053CD04B1D2FDDEE20
:1030D000ED4F5F14B26A50A5E02CE0527142F44B00
:1030E000D79B70509324884E3750848AE32E233B1D
:1030F0001F2C774CE7B63DF0EE86FD3C50E701FF14
:10310000077219E7E998B54CDDA2541D13533DA78A
:10311000D43DF27479F06AB1276D384D575BEB9C62
:1031200084FB66154EA409F311A0C04734F13F4D4E
:10313000E250421B3B68305F3EE00FAB852896288B
:10314000C6BB594D58600DA68EDDA4ECED31DF03F2
:10315000123D0D6C284F604DD3327F34268BB61A4A
:10316000480C7C4073865D265ACB6C4D7ECD100793
:1031700096C4FE008F32232C6CA0E6CA765BA64D67
:10318000E727895384E3003C7915FCE68DF7C29468
:1031900065CCAF4DC157FF4A9D164BFA5A9A1D7523
:1031A0000A5C7C9E403BD34DF4B8A2FBE4FA07597D
:1031B000A7D0C4400FAB54BC7175E04DF3D012EDF5
:1031C00005F9209E72AE776035DF7B290F5C044ED7
:1031D0003175C598CAFC7E2AA6527562634BA4104D
:1031E000F761054EF1D3CC4BAF61667FD0AB18EAE7
:1031F0006BC34566A9AC0C4E9558AEA0DAAA443113
:10320000A2DFA4317C448768CA1F0F4E5C5F73CB7A
:10321000C7118CF85DE5D72E0F0C17C34019174E58
:1032200020B37D8699DC2A332B99B184895252369A
:103230004CF6314EA8E3D97B81D2A95DEEB6C49C91
:103240002BC1BF419C52334E608C2DD151AFF4D86D
:103250001660D07EAD22E8AED206934E4B93454821
:103260005BED57BCA1286A54566240E57CCD964E72
:1032700066B487B5F2F7D0DF466CCFD77A1657F829
:1032800073BDCA4E8A4BF08093275C3EEB0F233D03
:1032900073D77978D496D84E3BE323F2B0768D116C
:1032A00034959858060CDF63CCC1E04EA132613EE4
:1032B0005F1399F6E7FE822BBFDAF43116C0FC4E9D
:1032C000ABA390BE21DB51D6E54B1CB71798C2CA01
:1032D000D585134FE3FF346A477CEE5028A466453A
:1032E0002838CCD970241E4F73494B58A88C84833E
:1032F00003D533BC3FBBC22228B92E4F346F44F5EF
:10330000B6337D95328C211B863238D5C8D23B4FDF
:103310002A7E6BEECD058626A108D97B509E31D63C
:10332000FB6D4D4FAF0A41BC71755FBDF5AE110825
:103330002160419C1F7C724FA755DD0FCD5C62BCA4
:103340006B5EB2E2DE2E08DADDDF844F36C5C226C0
:10335000295CADB7367E05ECCEE1A3372E05A04F34
:10336000D4F6B9EB6766B5C9D2718E03B929B37CBF
:10337000DDCEAA4F20CEDBDAE8E0738A87FEB21DED
:1033800013E631EBEC70BF4F539E2949709C785384
:103390004EEC2A6A76FB1255C2EDE84FB4ABE45905
:1033A000F0FE71C86089AB6F73C15AA0842FF24FD1
:1033B000CC4D69277E0CD362BEE938045FB58C7FA3
:1033C0001EDCFD4F0BE301F9F745E00963909D7B9F
:1033D00088FD7FA3E3BD18502E0B1EED415E8A4B86
:1033E00061AC17DEC4C470D3434D1D505362736C7F
:1033F00075429FA5BE7F215D73ED84F21C9423501E
:1034000070B050F15F4951E0A4C1C50F8A04248611
:10341000019A36501B99D553396368B0A6FACC1679
:10342000DF8034852F393B5026A2195C93231FE798
:103430002C5B3EFC02DBA4268FBB6550902DDFF792
:103440000B7A483828811FC9FD38006D8D259250B0
:1034500006B2844783813BB3AA69C1D58CB4E7FF28
:10346000C53EAB502899BECC959F4EA8B7A2798D8A
:1034700046049BB6578CE55023501544E8CC9E86F5
:1034800034864FC40A2DA40176D43751A581F49C0B
:1034900089233EB2A1B52EE030FCB377389E53515C
:1034A000FA0559FBB177A288237755AF1F3CE24A52
:1034B00082748151555EA2F4FCEE3E1A6425620FBF
:1034C000A84A781D20BB855100C340FAAD27964E0F
:1034D000A6CAA0F8576EFD2F1B6C8A51974E4BF66B
:1034E0000197590CF51E543579DB92D3932F9A51DD
:1034F00082FDD9D20F022BD300AF2649F4CD855BD4
:10350000D52DA05173538B64FA86BF373FF23386B3
:103510005C3AD0E2C70AC251E133A67213A58EA964
:103520007BDF731382C7A6879541FE518D2A738E68
:103530007A7E600811DB386ABA691DD22EB0075254
:10354000A8620CAA7535D4A3504A83B8E524384440
:10355000309D285297953B866918ED503C9644B6AD
:103560006DC9A44A08DC4D52330465846721A71550
:10357000779CF3B79B09CE2107525152D068824EF7
:1035800020D9356333BC0B37E105A69652DA545285
:10359000FC32BC7C41B651000BA0BA824FAC19483A
:1035A00038F85C52866BA9C3719887B2F7C08DE179
:1035B00089B0B9343B246752B82569DF0B1BF1FA97
:1035C00009E946A326D6E3ED8D906D52ED6761863D
:1035D000EB7A1BDE381B3C428D660DBD0D4AFF5257
:1035E00069E9CA66361B052F4B76475836FBFE1332
:1035F00037303A53AFDA9721B269660C612500354E
:10360000CC4538353DDA3F5368C3E69B7A6EA20954
:10361000F0222658F22F9AF0C3427753E16EFF57FB
:1036200045EC14E6A18E12FE638B5F63F7597A5363
:103630006E8833A7714EE7CFA7B613425840F20306
:103640009F5C8F537E9850A1E88B91E279F4CC8AED
:10365000A649168D0CAAAB5333AE45D7B493BE32F0
:10366000D5C0E7FA1E5C1955189ABB5341F03C16B9
:10367000665F6B7E748FF0222F5E8FD42DDEF75342
:10368000B23CB052496734A1612260AEFB16B00E65
:1036900097050A543CB8C3963C1AA9854AB4894098
:1036A000EA130E33091A0F546DC3E67A11763B7A8A
:1036B0008A626F78D4C427DCF8B11A54D8AF140FDB
:1036C000BFE89131DDC481DE64286264382A215468
:1036D000B8E0D156FCC04AF112E025CA3606018C8A
:1036E0004FA00000000000000000000000000000EB
:1036F000000000000000040FF66E370EF7220900EC
:10370000F55012005D110E71773D12FB72B9037313
:1037100056C61124B53408DA1C331262C65701D7D5
:10372000C61E107A0ED110090F70114F72D61132C9
:10373000308812969D801136E1460D472B32114F8D
:103740004F5F0F80F7A40E7FC5CE09D6213310C27C
:10375000C7450D0D89D612309AB60E097BA708AF62
:10376000E95710F23F01128A236B003F05E50C4038
:103770004EC20FECEA660F40B3590E9C738B0CD906
:1037800001CA11AE832B0F10D48107292DE5127ABF
:10379000CE411021BD5510836F3507867A5011C474
:1037A0000740116A484B10C4E6730E1C1D6A0F9641
:1037B0009CB80D91DDCE10876FD20E9E88DF10F37E
:1037C000DD4410F170060B21F26D1068059910268A
:1037D000D15D0FA1C07B043D837B0C0DA87512CC7D
:1037E00029AE09939A431050340711662D49106F82
:1037F000A44A0FFFAA160CD0976710FD0B4F034782
:1038000019F907AF4ED111F391600C34ABB01062CF
:10381000181200B428DE06532C5006E699B810DFC3
:103820003BDF12AA14B610DD5E06102834DE11CB81
:103830008A9B005306140C72315012C10AD90F49E9
:10384000E7150B2767260E863105130902350E9CF6
:103850000F5F01E020290E190131117846CD05399D
:10386000649F07F0CB65102DBD0D13A0ABC90ED121
:10387000E7A70E6A9F540AB569CA0FE1293D0AE21B
:103880009EC80C1D84910CEFECE50CFF6332121303
:1038900092C8104A12AF0D45445504515E6110683C
:1038A000EFA811063E2507E3F5E90D9C2C7D0EEEF1
:1038B00059990BD9E2471076FEE10F5D0EAB08FD7A
:1038C000EACA0F526AFC003A1E61121A675D12B111
:1038D000B19E0E812EE40F4B38F803ED59F80D0C14
:1038E0005668103AA2000D1E6E730DDF260B0CD722
:1038F00096F20C8520F006A89E1701B140D410BDA9
:1039000024D00D183639090AF24C13D51A730F9CBE
:10391000C86311677BBD0C600F870E1A5FA8013961
:10392000911A0EE368160FA97BCA0FD42B4F0E6CA9
:1039300021D80FCA71D50E87A3C11063EBCF121225
:10394000EE0C0F30660712AEFD5912D0E0AF1173C6
:103950000CA40EF5E29D10957BE612A8313D103BBC
:1039600008050F58D2C412195A2710C185EE074E08
:10397000D803071C537310DD003912F9CD840923D5
:103980006107102C6D3E1026A81B11F7884E108978
:1039900000B20674367A0C2CBA7D10C08F300F61DD
:1039A000059A0E4591210E1730390E3E88E211140A
:1039B0002B5811E3CCD30E56FF7C0D36096110C392
:1039C000421D0FA0EC930B88F13E10EA785210A62E
:1039D000996010BF886D0C1572EA0BB4EEC210121C
:1039E0002B3D0D0AE0D1103342491088BCC0056858
:1039F000EBC811CB937F0E4EF7AC0E4147010D1172
:103A00005CE70E7C70CF03EC3C4B092BC7790FAF02
:103A100032C711F6D76002E67CD112F88DA50EE50B
:103A2000656312F9D16602C87DC20D5FA0250F5DE6
:103A30001F1712DC66C30CBE39A80954536A0E7FE7
:103A4000EECF04C8746C0B519086065EF3EF042130
:103A5000A1AE1274B6091347A7BA0D07019A10B4A4
:103A600031430D513EF00F73076A0F02F2C210345A
:103A7000A35F004ED1F30CB873C10F058805101079
:103A80005E180D5361690D3A27E412789C000FE728
:103A90002EBE10C1B5130FF5BE070D6967EA10A859
:103AA000DDE107AE47A80FD6AFB511E3538E11186D
:103AB0004993111C1CA008B8BC2912FF728509CDBE
:103AC0008DBE0F663A3510FDAFF70E2B575012B072
:103AD000B071102E47230178464800A155D510C07B
:103AE000CE500F321FF309B587120FBB91E911A910
:103AF000B8200EFAD8EA108B643B0DC73E2312C6DD
:103B0000AD00129885A911C7C6400DE8EC730ED31D
:103B10005CD50E7B856D1272C2D10EC6680209C3D8
:103B2000B1F21113DAC0112F8A97104AB50D0AAA03
:103B3000D9560EFF21F803202EEC0CFDA3690E438D
:103B40000AB41211B4BA071E684B09D97C0210EFEF
:103B5000A65310BCF8B40DAFAFFC0E5B52FE0F6F56
:103B60001AB10721B7660738E47407B004BA0A84AB
:103B7000A5280D5D91970F4B14F90C71365B0C194C
:103B8000A5620E814B900F11C41B10C61B900EB086
:103B90000E2D06BF4B810FA0515007BB7CFD0D833E
:103BA000C7490F2B689600F813780EF5A83E1052FF
:103BB0003D990FC870740E4EFD990142AAA50D5E85
:103BC0006B5E0AA6F27F0CBDB57E0F08A7EC0F094D
:103BD0007A980FF529AA0F854F6B0E9453FA055C5E
:103BE0003D9A06154C3D0EC4F90A036089B5045E82
:103BF0000ED90F95DD0A0F1890230D2B9BC30F0EC6
:103C0000D6B80F2CCADE021A7A700F1108B20CCE89
:103C100013E3101FB6AB07C144870D1FBB900CEB1D
:103C2000C53E0D7EA5290F9727F20F3D8A4F0F88BD
:103C3000ECBE0D95DCF1125CED2510C0203107C8FB
:103C400060FC0F6FD5D911845C830469F17A0FBED3
:103C5000BAC30594CABE123389040D4F28580E18F2
:103C60000A02134D66C410C585DE0E5944090F7152
:103C7000096A0F11D87B13799D4E0F9BCB5B07B55B
:103C80002DC1129D0BB212BAB5750D7FF63E13E72A
:103C90000B500AC7295508CA775A0505579A080CC8
:103CA0005F780CFA55B506E0F6340F704C89048F36
:103CB0006B5B10575ECE0F96FD470031759B103D34
:103CC000A495045A5ABF07F69141102BA1AA0DC919
:103CD000C2640FD47EF90FF518580D7D984D109CD5
:103CE00081FD1191585D11F0D4EA0D5303C60FCC3C
:103CF0001B08101455400D00E3A808D094D50BC440
:103D00006D780DF637380BF7656F04E934BD0BB7E6
:103D1000B0580E08BC810CDF3A860ED1AD2610FBE0
:103D20001E12103EBF4A10FEBEF30FD73B2B1014DD
:103D3000EE4208FD574C0CC0434310022B59112E84
:103D400058F10FCF1E9E0F7655F70F19FB990FE50F
:103D500027BF08BEA26710FB46130BD0768513322F
:103D6000542F0EC1BA4F0CED0E6C0E876FDE0F3064
:103D7000856B12EED3DF0C0FB7A70E441DBB0C8D65
:103D80009B310F2B731D0CF2E9B908AEC91110312C
:103D900093D911430CB9007095581078FA5D0DE86D
:103DA0000EC5106A4699100AFE950B21724A0E063E
:103DB000E6200EC76A9B0E6F0EA1106417A30B8638
:103DC00079470D9A386B0E89E5CA0B78EA740C377F
:103DD000F82312EBEC3D0B19198C0C84359C07A7CA
:103DE0008F440D149A800B90AABB0F87F2EA0D57EF
:103DF000FD840DC0E8DF0D959FC20A9E886812EA17
:103E0000B1550D5B62A20EB9C5150E7EDFAF103540
:103E10009AFC0E5D4E800E091E5212D034270E3CC5
:103E20009D6A0EF3A9F50F954DDA006D7D7110FBBB
:103E30001D6110448C99105AC20512AD8FE40EAF6B
:103E40006A021189C1A10F7D1A461068FEB8129E40
:103E50009CE30F73C7E20F682C951027654D0E8900
:103E60002A18133AD91E0DA03BF41025A4040DB353
:103E70000ED7111A38840C3B0A160E8B253B0E0DFB
:103E8000C1F20FA6DD0313C1901B099F3CBC0FD5E7
:103E900083750D203F210FD75BC30E1E71C80F988D
:103EA000B4E30EEBC45C11F11F580262451E0EE430
:103EB0000DC609D6CD9D1007FB490E34913F10E485
:103EC0002FEA0DD95C6010CBF04D10FEC82A10F21D
:103ED000C93E0A8535301184E67A057BFE0110253E
:103EE000D0AF0FB3279303F36E280F3D16900D72DA
:103EF0009E570D4A39010D9AEBA411FBA2A10A6647
:103F0000BA320A65D60211F3B2C211CE924A0BAE92
:103F1000DA9C03A47CA400781EB60623008C0C490E
:103F200063421079EBE30EE1FCD10E38380A0FDA68
:103F30008D2E024CB24F0C4C517712AB0ECA0FA70C
:103F40007BA6104626570FEB8F760F141BD30F98C6
:103F5000C191105BE17A1047B9000DBDEC2E130F33
:103F6000DAD20DFAB0E40E665CF50F0CA18910DA16
:103F7000CA060473C26E0F69FB66110188200784AC
:103F8000C28911CF5FAB0D6523040C53ED8E0EAECD
:103F9000897F0EDA867403132DD30FC7891B117620
:103FA000B5A307A6B6F30B789D7D0B5FC9A2018769
:103FB000E166101A388D0ECFA780109BB8C2128907
:103FC000DD2B0D2AA079104B232A0A00D3D204FF3F
:103FD000CF920A2583C8039639E40D92D82110D9CF
:103FE0009E7212C2FA460DE48F1E1099C67F0A8592
:103FF00028F412205B251272D460092BC4520F7E64
:10400000957800B8FFCD0FB3C0590FD2B19910FD0C
:104010001FC911A83EDE0F2984B60DC9C2870F4003
:1040200019B8123224CC0D4541920B53414E06B1C2
:10403000C5A70F3D7C5500130BA01245DA7B0F3D41
:10404000D2E30D12DC740E6FF5E911B697D20FC2F0
:10405000272C126499AE103FA0B810A46070059E82
:1040600000000000720FF66E400EF7220900F550B6
:10407000120061E27E8A5CD3838B5740E9453FF8AA
:10408000A9D2C161DBCE7B6AD91D52D297625C3C5A
:10409000BE89293744DE115D4D7FC701F25EB7A1AD
:1040A0007961A7F3479BDB0C51BEDFB5487C1FF558
:1040B000900C0D1A1BD877E108839FA37CDAFC6D66
:1040C000B379FC06D5A21DCA840864FB76818425D9
:1040D0008940BBF76D2B2D0E3097E5B6D9745D6A1C
:1040E0005D220641D4B4AB73DFDF90640F26B63196
:1040F000937CF463A41574843E3730F499EC3A5BF6
:1041000030C4D3D56F26E0D966E86AA5A4EB696E02
:10411000A947F86BDD3A8C88DB5B632ADE3DD881EA
:1041200014BA1243A5C4FABBFDC96779B33C092888
:10413000D04BB6E1A9862BDC2E73FFC80FF92013F4
:10414000F8AB3CED383CCB0BE3D1FE0CBE76AAF1CC
:104150008CF501272E2272ED477978095802DB93FE
:10416000F49258F5FE4F6E8598584E2C2CAEA45EF6
:10417000A3D60F452D00BAB7F26C797FD0EC3F245F
:104180003F1443E01282A5F9F95F45DCEBE055AB43
:1041900098ECEED1E6D3408997CA544C6E32D737AB
:1041A00061A3D4CACBA529B87591B7636C27C13870
:1041B0003BEFE7D6796837A2FDAC926B206FECF04D
:1041C0006BFC7712E336DE17831416F046E83152A3
:1041D000F4417A295CFA5B086C9C1C3117E904DD18
:1041E00075EF5835984CC824C2E0C5106CEDD42A40
:1041F0004E268AA794B476641C1D9EEC837C8C3C6E
:1042000092656A2E08B4465CD8DEAAAADF98F2AF9F
:104210003402F80F6BBBC361B158AD0525E8BBC2D2
:1042200036674F6DF8DE42BE69602084512ACED1D8
:10423000B3EC49030AE7156BB0FFA308D5AD895865
:104240005A32EDB67DE1263E450DFA96028B38B81E
:1042500023A1103C9F2B68B6593A04F0F771B39F25
:104260000FF6F584FE147202749FAD5CD169B0B094
:10427000E99EE0AE347C32CC1AA0DA8C6410443370
:10428000E6EEF08979328C068FA0DB4A1720399749
:104290000F0000DF6ADE569EEFE1B623F1DAE3910C
:1042A0000D3B0AAD41BF4173435619907B64B60183
:1042B000F2F490A8017750FAEBF6114836A57C226B
:1042C000B0C74993AF3139690B90923B43B672C77F
:1042D00081C6FD3286E01547FDA5844C2642065A6C
:1042E000DF9BCBCE28829F42EC4BFC965C0AE139E7
:1042F000989BF0986C462D2137C713A57347097317
:104300008F63C4F6604DFFEB71C598865D8FADE697
:10431000E17979D644B73B2FEF497035D20F24D6D7
:10432000A5B3B3D0C92DB8F6196B9873EE6859765A
:10433000B81D10EF3A2EBB65EEF80F448CCE51EE4F
:104340006F0FB5BAB0F96CAF8496E27AAA9500F314
:10435000A1E1D3931421893679CAFBED24D2F486E6
:10436000D82A472AE14AA728F1365B003701EB74C7
:104370007CF0CA3C7C5C116763EE82CF7C983A1972
:10438000293100A154B6FDA8CC8F27D0F3ED8D3B89
:104390004C7F689776D13ADCF1970B96C85760D37B
:1043A0008F669D2E7C7491714F270E477B03770794
:1043B0001BA77B5D8ACCA5C28FD76D64A02604485D
:1043C000B9FA7BF62DAA2CF0A49DE3968DE2079115
:1043D0005B242458C7BD44E5072D65C87A8F6E93CA
:1043E000DEFD7B6AD91D52D297625C3CBE892937BB
:1043F00044DE115D4D7F0714D584AAE826A44D61E3
:10440000AB61C2D089C081E998660C95C86FBC3693
:1044100094E730246803135C7B9148E77BD9F68AE4
:104420002A48C08B2A277E579A513E63526B7D19CA
:10443000A50734210778A8FCD31DE295E6619E3CD0
:10444000D9EC2919389CFFEB71C598865D8FADE6D4
:10445000E17979D644B73B2FEF49AB3117ABD4B7ED
:1044600085FCCD176AAD1BA1D3FA8EC83177BD8DFF
:1044700099D64656DE50733BF89F1961F56AABA496
:104480009C4EE00193E107B217FF6AD8C0AD3B1222
:10449000524E3F7553BFA5DE9ED5125E5ABA11F536
:1044A000D5586ED501E246E01E16CB1812EF827386
:1044B0005D00B1874DC196D37C65FDA5A3BEBD2926
:1044C0007D70688FABF362D30F09FAC82D22E883A1
:1044D0009AF4243E55385DA052CA74A0BED59443C8
:1044E000C0A6225F5ADFE7D6796837A2FDAC926B8F
:1044F000206FECF06BFC7712E336DFD1293B2AF01A
:1045000035D3366E5AE52294AD799C844E79C60730
:10451000D3AD6583B1C4028E4137FC752777CFD503
:10452000FDF32B5D4872C504AB8F4BC40888FE5B5E
:104530002B0554CE5B1241486928AC0F8F9E2F0D7E
:1045400093C27F9E1EA68980AA65A47D37EDAC3DEF
:10455000E1FFDC0467881AF946076E4DAF74DA266E
:10456000910DA029F8EF7C0CD80540716B0EFEC1AF
:10457000A3F7D68F700CFFE17F7F4FA1001543AAF0
:1045800036E1085B9CB19AD7D6A957307EC060B897
:10459000EE1EFEB7C6CCA12AB88244CBC0C5C1E28C
:1045A0003C8CC293ED365B4ADDC1BA59E3F0243D41
:1045B0007C059E96C410D627005B786D0D23995A12
:1045C000ABC5BCD801A278640A2C84650FC5557DA3
:1045D000EBBD4123D10B07951C040E3A66D4631E34
:1045E000122A0DD679122AA53E413DC76F6F4C00A5
:1045F000DEC74FF42AD6BBED571AC19DDA8864771F
:10460000F5F5D9FA533CEEB3ACFC2C1F8A35E21415
:1046100065C20F80E99F79E3F365615481494C5A83
:104620002A5AE22C944878EE32263D8EA0C01368B8
:104630004D07AF58B5097DF495DDC25DEC7922F4E4
:10464000B83724CA697E1773D51736615D6A7F0053
:1046500006AE1640BEAE7E58A29A34C41D117163D8
:104660005ABFF2F4C5F67B84AAE3405813C0203C3D
:10467000A27967877736C431C211F025F9EC4A1068
:10468000A39CE21B6B5665962901FE363BB3B29E96
:104690003B494F9FC406D8ED6CDCEE9B8EB15CEFBE
:1046A000291653000C65FDE3B7F186BF6015595616
:1046B0005514782EC4CF9EDFF76E27498239A48A1D
:1046C000FBB87337805EDA4A2BA4EFC8C53019CC2B
:1046D0006AEB8456F6D2B106796EC3A41BD4EF31CF
:1046E0001A70DF557EF3DE5D4A90F06D9886ED40DE
:1046F000408CC8C1FBFA5B088591C26105369C09F4
:1047000017BAD73761A3D4CACBA529B87591B763B7
:104710006C27C1383BEFAD2DE4E35E212977EC95A2
:10472000CCA26067B723B13CFD6B03BCAA1508841B
:104730005532960812CE84B1D052A7E2FDD9BA27DD
:10474000A0524E8266FF806042508B4D1CA5F6BB86
:1047500062448C9629AAED3AF5DFF3AB1910FE06F8
:104760003181D953E4E44F7B1CA45796846ADA5E06
:10477000105279D99C03165C5661813CDB1C258163
:10478000EA5C7083F02049A65822171B4636B8070A
:10479000C50F86A72EBA340D68C19842755D030116
:1047A000322716C0F9524608CF8907F39C10DD4E18
:1047B0000AB25A6000CA29540E5A00DFA603628565
:1047C000A67DF4DE172839749553D282B16FE625A1
:1047D000EF36EFF08C1D4E7AF1FB6B78AC6C57AD79
:1047E0007280D0D82FA00546EB276AA018D10725E4
:1047F000517C15C91CD25457F2321FC21CBC4380D5
:1048000017C719F59066168619CD56D74D93A18115
:104810007F2FE0F758741730FD43280FF66E480ECF
:10482000F7220900F5501200675D02896EF5001548
:104830004C500625F61D0B7532AB007195D900461C
:1048400048A003DECFE3009E106B008B605503BDD4
:10485000C4A400DEBF3F03F152A000C261AC02500D
:10486000999B01DEDE5503A9284703964AD1031020
:1048700009FB017EB4D3007A40EF01FE8E9D039BBD
:104880003C07027706D801EC6DF6018DF1FB0022A2
:10489000EAD100C48CF700D198FB0077F12701D250
:1048A0000FCC031E21C7004395970385B87B020DEB
:1048B00075E0021F6CC3026412F8001C111903DAC0
:1048C000394C038ACB1903D110EF025838F1029109
:1048D0008224035AA70D030C6EF500157F9D02512B
:1048E00071D500926F0904AB2B260313B87B020D20
:1048F0001FDB0AFB63580287861503CF6607049FF8
:10490000C6620607C51204341CC901C928470396AC
:104910005F24025BC2F201EA56E70129F46A04BD92
:10492000BBA90306EEDB04AB941B06D9EBE501E75C
:10493000E42302F5877F0354EAFD001DEE270225DC
:10494000BF66039750F800072F32022358EF010487
:10495000017C0342D2E901BD30CB01817FEA03E251
:104960008371032AFDE2015F0202025B16CA00C7DF
:10497000200902F395EF01D1DE5503A96BF200AFD8
:1049800010E301F14CC9006840760035130502665A
:104990004EEC03A4DFF103B2923802D320FF0141B1
:1049A0007FEE0075DD87032DC42602917FE5018A25
:1049B000BE0FF66E490EF7220900F55012006A008C
:1049C000C6B3E456250156051CAFAFD27CBD8CDBC7
:1049D00099EC8200E2F52DE84CA2BC7D26AB9BE46D
:1049E00026A2D5E32E2F8600637829961C636F8F4D
:1049F000449E3D9209E0762DA81B86006378299697
:104A00001C636F8F449E3D9209E0762DA81BC90060
:104A1000A845E9FB4A9B2D005F81EA7F0B781C02C9
:104A2000A97C6401F7441325FF23C4754B635AD74F
:104A30007AA115BF893BE001621A9CE0B7531608C2
:104A40002EB7F0F26CE91CBF711ECD02ACE42E94BF
:104A500012CB8A5EC7A90A2E395F6A964876DE02B3
:104A6000FB58F937E5208CF36DCA152CD6A057DE1C
:104A700062555604BF4742560D9B4C4259988BB124
:104A800036C2A2A2F5A66804F592C5C317DEB4B477
:104A900076BA9310E00FBA465754E6048E23C050FE
:104AA0001E8CB530FB530BE62F69374A9D7FD60528
:104AB00054A507221E0ECCFDEC8C86D527725FBA5A
:104AC00026444606AF043BC6205D54A65B61BC0687
:104AD000E63962693FC13907BFABC2B82065D2BFB2
:104AE00041D340445FF98019510B42077D007B762A
:104AF00089680BD68474B8BCACA2223A675ECE0734
:104B00002999D416455BF6F50BFCFB3309BBF44041
:104B10005EC4CE072999D416455BF6F50BFCFB3332
:104B200009BBF4405EC4DE07573180D56A73AE51CD
:104B30001492817A3564023C41B6FD077385845432
:104B400030931208CDBA3DD689CBDD82DF790C08CF
:104B5000B51D432AC5F5F1B6472FBF6DBC7ECFBD4D
:104B600020C87C09D74F5C86406ADDA978EAF559F0
:104B700083AD801E01881B0ADFE8A2435BA512A556
:104B8000DEB7513D8BE97D30DABD190B909783C6B6
:104B9000E971D8C0EB16B381B85C2A6A8ABB190BDD
:104BA00027599420D3182B71DE7F602418F0945479
:104BB0008014670DF62A1E80DC63AE59E8821671F8
:104BC0002B7AD5D0DB83670DF62A1E80DC63AE59C5
:104BD000E88216712B7AD5D0DB83B60DAEF84BEC9C
:104BE000F9BD662CB382A9D576C075F284550D0E39
:104BF00051528A1963D2852AFB8F52CFA47A9FC261
:104C00001021360E73250027F448F4ECB2951E955A
:104C10005B62B42F25C3AF0E3EAFDBB23DB808E0F8
:104C20006B72983B9A79ACBEDC3CBF0E2B4D821D5B
:104C300067C53B45D4F4A5C255FD4C15EF121E0FB8
:104C400088C4CE47ABFBAC8BCAD8BC1654B78AC855
:104C5000B9B51E0F88C4CE47ABFBAC8BCAD8BC1607
:104C600054B78AC8B9B5341152A67B861933FF648C
:104C7000BA0F87AF5FE0B88E0439341152A67B8635
:104C80001933FF64BA0F87AF5FE0B88E043937116C
:104C90001BCE09648D6DEB519E9CE618377614553A
:104CA000EF477811DE2A892FE5190A071348ABFE72
:104CB0005728BC139DD7C7114474CEE8827FACDA65
:104CC000E401BF03ABB29886F3E54F126F5E64D088
:104CD0007AC7EF5DE6930661D0F5C83B87CA7112CB
:104CE0007D73F60C134A46BF986BC39DD08B435B14
:104CF00001DAAA12D79AFB36A6C03C3A8B14531796
:104D000032609840FBBCF112834EAB33FA06EF439E
:104D1000ACECD0E6503F475CAB5BC913DBD7C18A34
:104D2000BE7F97208BD54E9F0CDF4C30471F3C1425
:104D30000CE832FA6C36B64859A07B5418053B870C
:104D40009855CE145E77520F2D099BF42D42F8B87A
:104D50002BBA63B0E0F331150CC9F6E00F8A198362
:104D60006C72A8FB6B1BF3C7B2A931150CC9F6E036
:104D70000F8A19836C72A8FB6B1BF3C7B2A9561577
:104D80002FA9D5E7B7768FE85E5FF4D36949D85D80
:104D9000E9EC531659FBC44CCAF9E449DD1D7E9D6C
:104DA00013BAB4374978321727FBB44116D5B7AEDA
:104DB000C34675368692128B0601321727FBB44123
:104DC00016D5B7AEC34675368692128B06013217DA
:104DD00027FBB44116D5B7AEC34675368692128B03
:104DE00006017D1703D8B88BF6B38FCFE373F39129
:104DF000C7207CB406D1B5179824DC9A4A471641DF
:104E00004412D776300D546BB0C0E31761284AEED8
:104E1000D486C80B72286B219CF61D4A44D70E1805
:104E2000E4B691E0EA3285310C3191C3E1B5D22A82
:104E30002A45471805C7EED1A9CD94B517B045311D
:104E40002B0C0F7D44009C18F849E6BE9F6EBFAA4C
:104E500038F8A7336E0B9CE46997341BE384B8C51C
:104E60005A4D5EFE3178F32AA84B48CD7788C01B97
:104E7000CF2588F525BFC526E6DFB1B3B4360F3B95
:104E80004908041CCA9ADCE3C5791084BDD19BAFE4
:104E900050B9288EC519E51CD7AADEF98F05C47054
:104EA0008427600C60319D68D5B2101DB7D7505D66
:104EB00083BB90AE49E28D6B098988D32027111DF1
:104EC0002EEEA722D4213875B4364A559FF19FA003
:104ED000C627111D2EEEA722D4213875B4364A55A7
:104EE0009FF19FA0C6279B1D3881BA3EBB6C80599D
:104EF000DBD94923152662E25245371E9A5E0D938F
:104F0000E11B79AEA25B4F1161BE04585ABD381E39
:104F100039E3F462A7AF9317888850ABE9D90E1331
:104F2000D0E1701EFBF7453490803D228179C604A4
:104F3000F7AAAA0DB7E4A81E4D3FCEB46E8856EE70
:104F4000FA2F0ADF02C8868E6917A81E4D3FCEB41D
:104F50006E8856EEFA2F0ADF02C8868E69176D1F1B
:104F6000D8FC7AB66E7BA7DAF466C9A295DF3C203E
:104F70003B1CD61F800A68A21DC036B1FE327EBB24
:104F8000145B281EBF5CF71F5EB012DC1EBEFAA0C9
:104F9000DD92F48DCC8478237D8A47210F267F1DF6
:104FA0005A5A68BCA3268CD5CF199399778FC722FC
:104FB000431BD5E47CCF2E7C54A4CC5766C2FBB1F6
:104FC000D0196824BDF41ED0D2AEBA9FC5961C710C
:104FD000D213B59B8977EE243DCD640E73D3EDDEFD
:104FE000373F4E5315A02A7B975413265DC1F1A27B
:104FF0004F18B94F290AB4DF7AA2020B50DF60269E
:105000003BA9712398DE52AA58C9CA16C9D6D4A2A0
:1050100072DBC8264ED282E763F47BA265CA4504E0
:10502000FBEEB6F30984F7268116955487D119B59E
:105030009F9A28F0A87C32C2ACCA79278BDAA338B1
:1050400095C9B7C96B5872FE334F76514C9B0428F3
:105050009543790E922C5034EF3BF77D517A3EE424
:10506000234704289543790E922C5034EF3BF77D6B
:10507000517A3EE423470B28281862D620388568E9
:1050800029504BE26EFC56D808B47028084F3F9B5D
:105090002FBAEDCC026C7972396F9C91150D762880
:1050A0009E7872D4E2ABD2DD52E7E2CCC6DA395A4E
:1050B0000C610529C14B28750AF2D06F5AECB82053
:1050C0009D2D7C38BA76AE29F00680B42023D49288
:1050D000A0163360464213E6548DDB29E8E1E899D7
:1050E0001A86DCB634797BF9F9070A734D412A2A0E
:1050F000F30392474D7F54DDD2AD7891BC3ECF553E
:10510000A1E4052BF8909D6E161E750D1AD8C75890
:10511000BE62574298013E2B21893A0275E5975F9E
:105120002136AF43401BF6171EBC712BD926BDF6A6
:10513000F504C9F74591B06618FE39F3827F992BC3
:105140009EFA9FC4B96D383B40C46EF372845A1402
:1051500067F9CD2B232D810D72DE26CE1D47E199F7
:1051600002E7CD75854C022CBE62E1E4EC143248B6
:10517000BEC3532CE1B7C30A8458E72CC520BD3504
:105180006680C38591CC0B495813BB76F9E46C2D2E
:1051900029630B210B0A4CA0C671ADAFB4224B5B47
:1051A00042ACE92DE3FEBCCBC8E541E0B293BC7B49
:1051B00024F582711D291A2E0CDEA43EE969EA0C41
:1051C0001C9F4C0FF4100C35F2ED942E4139885A87
:1051D00008EF840D6893948CCDB133E322BC972EF5
:1051E000A86451594C54F5CCB2671D7355A8F77596
:1051F000954B972EA86451594C54F5CCB2671D734A
:1052000055A8F775954B8F2F46DED005834068452E
:1052100080AD6045A7D9DF3E0628942FB9D8CC478A
:10522000B53845D20C6C5FD24A28CC693D2CD82FBA
:1052300010962B7E6457AC55094E39C53C916B4D89
:1052400066CC0D319586BB307F27D55889DC682721
:10525000FF76A9A16C4DA931121F4EAD905920B116
:105260007763D9BE3071D3564B78203281E15780B5
:10527000029F7644F6E95514A69F4A2553A32A3285
:10528000A38D2697A86AF2D60CFCAB301BBE0CEBA4
:10529000AD775A32516C36ECCF8DEDC98DD5DC5CD3
:1052A000319F5F62F27163323DC181EAA200395BD6
:1052B000D4CE3080F8CAB413D96563323DC181EAD7
:1052C000A200395BD4CE3080F8CAB413D965173345
:1052D000C29F509D4CF802AA095C5226C5AC9E0F95
:1052E0007AA48C338176969C7DD43312DAC82BFC59
:1052F000141D3A71796899336A99B6455A8CC1FE82
:105300003A792851948C2BD48483BA33EEDE403121
:10531000C86659511F8FD3A035FA4B7EDB073D3449
:10532000195E8DB2A2CF31CA5E27F2CBA015EDC9AE
:1053300036A27534EE1DF544AFF823AB2803400ABE
:10534000B7E6FAADF9D3C33492CC1101A9CC3042FF
:105350004D456AF464B9693314D5D7341727F2047C
:1053600062B72803A0C12554BDAA2F094BEAD43542
:10537000A0BC15A175F526EF58A86F426F17FBAEBC
:105380007011C03681580AF3D07C95ACE8EEE78204
:10539000167F78D94286E936389C021B7355CD7743
:1053A000D590B0D1D3136CB5019FE936389C021B60
:1053B0007355CD77D590B0D1D3136CB5019F4537D8
:1053C000395ADC017E6872AEAA35BBEEF9E8E7C94E
:1053D0001E221E380C626D2D900F4877677942F1BE
:1053E00035F24711DFDB0539CEBA3E8894A3032A94
:1053F0001C9D65A868EB5931293A3839CF0ACF236B
:1054000065FA9256C0E9910A365D5BC81A0E733A86
:1054100075F211E94EBBFE51B82288327446174D21
:10542000C475883A693357F1450620AB201BA7376E
:105430003BC369482B20D03A82206CF83947ADDA5B
:105440000BC119A775926B50CF15503C2F34A7464E
:10545000920117141AA2FCE84870CC31DE11153DF8
:1054600063A72E0AC249A2C722FC5BBF9DBBB5CC75
:10547000DA957F3D8C9E058CEA8E13C1BC02AC2B65
:10548000E624AC4B4F380D40066F6D5D36CF07A656
:10549000C0648854E541E4DA10C23440307B8E6742
:1054A0005B650BFD0F5D82805F721481FA44C4401E
:1054B0001EB4FC15233BB9BC598B0CC0FC430E81B8
:1054C00026862D41D38A3EDBB8D2963970DAB18F69
:1054D00033750B3985A99941A7511FD3115F749971
:1054E000B5AF67BDFB2D336F728A9B41FE9E7D7CFD
:1054F0001844BC7BE524BDA5253E1C463E57C4414F
:105500004B0B2F24323164DCF6CBDF801B073D329E
:105510002938E041802DD98DAC42044E535D009076
:10552000E3F702B3C2AEE041802DD98DAC42044E08
:10553000535D0090E3F702B3C2AEFC422C39201C4D
:105540001FFD5468A3FBBC7421A870E2B98200431C
:105550001AE336B6DC9FC9B200BFB8E55296567161
:10556000CEB80443223C035D107E4B1B7133914E39
:10557000ACBAB0BB100A0A43717F6526EB02ECF6A9
:105580008D60D5FDCE1802B6A6100A43717F652640
:10559000EB02ECF68D60D5FDCE1802B6A6101343D3
:1055A000716CBF0C2E1B9D9576FACA573CEE14D336
:1055B0003B3C1343716CBF0C2E1B9D9576FACA576A
:1055C0003CEE14D33B3CD943966D0988D0DD1FD403
:1055D000C9D4602CBB525B54E4D5D943966D09887D
:1055E000D0DD1FD4C9D4602CBB525B54E4D57F44BA
:1055F000B3C1EDC5CAF76C095257EBCA711A6B8B70
:105600007FCA7F44B3C1EDC5CAF76C095257EBCAD4
:10561000711A6B8B7FCA4645807B1242E3438EBB77
:105620005CEBBBB6AE2C667CBEFD38469EA0CE9130
:10563000CA9C7B2ACF922AE572B8E663328008477B
:10564000E963D41341A58F302B72C7CCD5451D61BA
:10565000F5053947A54FFAF45C82D0D420CE9BC320
:1056600049A2757FB2BE3947A54FFAF45C82D0D407
:1056700020CE9BC349A2757FB2BE6147E844F0A724
:105680005325ED93A2B0E6A547C745532065B14722
:10569000D7BF7930C1F41280F5B65D4690A289C8B3
:1056A00042981D48AE663183A2B070A80900E95F38
:1056B00094752E7E4985294889CB977C0CF1B38758
:1056C000D86B6C900F8353E9FE858048B51E1F513F
:1056D000B8A52A67EE3B576408A81BEF5B927B498D
:1056E0007D36152FB0D978FA71096CE8C1F9DFAEB3
:1056F000440F484AAB46B3ECEFD37A900D483A13C7
:10570000561383F66A26764AB6534D81CC155075EA
:1057100032BB83B3365CC60626BB764AB6534D8190
:10572000CC15507532BB83B3365CC60626BB7E4AA9
:10573000D5937F37F1DA7B59CBFB2C52A16AA7F0C6
:105740007B66884A8BDAB4702BFB2A74B4E60FB5FB
:10575000B87AC46A58A95A4B5FC9938B325FF5B4C3
:1057600024A0B3EF580AEB7FE8AC804B894F39EDAA
:10577000B4538A699A13FB3D22A2AE819C441E4C0D
:10578000D4F946E7B937AF9BBA4BBC8A5C94302456
:10579000E4ADB14CC547ACFD5E0DFF1E3B6E90F510
:1057A0008F2038EC6CA1BD4C6EB9F01F024805C5C6
:1057B0007549FA1234AFC5E6C7F0164D8F2B26B0E7
:1057C0001636ADD800B3D1704C9B12C405BBB14D99
:1057D000F10E62E242A853E819DF7B6CEF264A58CB
:1057E00050B0C84D127ED81787A7F0E15773E695E1
:1057F0009EB515F42378C84D127ED81787A7F0E11F
:105800005773E6959EB515F42378064E44EF9D52E6
:10581000C07D30EE9F773F525A3FB4C1A4E5734E2E
:1058200088BB04485F7978C5FC3919880B020D677D
:1058300062D2F34EC263ABA894319329F4BDE21057
:1058400090BA9120D559314F4D46C9169EDFA1D04F
:10585000141F6B0A653A8737781F325147E477E1A6
:10586000B6C2D04EB47A2DAC12B2B7D27A5D3252F3
:1058700067EFDC06C3F08B33D26596BFF6A0911CB0
:105880004A1F48521BC67256DD46FFD4FD96D1D042
:1058900017100D610852645226F0B34DDF06F4185C
:1058A000E7A962A74A8501717C547F525867225646
:1058B000036E59C86190D4EA42943996F8167F5223
:1058C00058672256036E59C86190D4EA42943996BB
:1058D000F81661548022C9DA11B21F7EB6A0EEFA22
:1058E000E06A3CC9017261548022C9DA11B21F7E9C
:1058F000B6A0EEFAE06A3CC9017248551EA733A66D
:105900001A12B4C14B8B13C36F48397C63DE165631
:10591000A4BD116FB618BB76F2200F082443A6B1C0
:105920001208915618E6391D60997A859EB7FE5780
:1059300060E2621BFBED7157805D3C1066F6F3D1AF
:10594000C33B94D58271B4E398549C58A8EC2B6D5A
:1059500057BB1B7C0FEBE17DDDC34DE44A736C0F3D
:10596000F66E590EF7220900F5501200351009584D
:1059700018D210AE126C06BD126C06BD9D8E0C3195
:10598000E56D0289EBA9012F00431229A9B3027D1D
:105990009D830347A8B60A8408B30B8507310861C5
:1059A0000CDD104680C510939643039D6E1309C00D
:1059B0006E1309C0BBF10FBF4047027BA65212769F
:1059C0008CA0122A04B4120238850D79EBA212EFD2
:1059D000EC011010EC0110105FB31082AB310840E5
:1059E00082A2050452FF118FBCA412D8C2C210D9E2
:1059F000C2C210D94384064043840640BDC6044C4D
:105A0000288E08D325961170810C1272361D0E6BEC
:105A1000321910855AFE0A4F870511BB5CE20B2F25
:105A200031170FDC7B4705E87B4705E85764102CEE
:105A3000F20510474695041D4695041D4695041D24
:105A40006BC40536BE070CE6F2790234BF57106E00
:105A5000DF610D10F3C0110FCB7F116322990FB7D7
:105A6000D7CD0FA4C7EB1039C3E50FE5E8320239F3
:105A7000E832023990A80E187C7B13F992DA0C9F59
:105A80003D0908F969F110B769F110B76CCE11380A
:105A90006EEA11B189330994BC81117AFD790C0544
:105AA0001FC6124F82CB0FFDB9AD0D6204DA028919
:105AB0002E5A023BF62B0D642FA70DDC060E08BDF7
:105AC000060E08BD5E7E01CCD4BD0816B08813F367
:105AD0001C0113EA31490FEB26BC12E45C5E094657
:105AE0008A5E0522AEC2045117990C390F5B11C7AB
:105AF000DB5912D4C81511960D840626C17D0F02FC
:105B0000219701595B56026994E6051B35D212555F
:105B100035D21255B1F701F913B00B683D7C01D5B0
:105B20000C1901CC1D4A0F6E06DC0C6E45A1035901
:105B3000957802BFB5270F6EB5270F6EBBFA11E23D
:105B4000813313169B670D255D050F9D31B100E96B
:105B5000792007C11BD90130E0B1080691530D71BE
:105B6000C5CC10FE05A80FCD05A80FCD187E0702E5
:105B700052CB129CDFD20B18E251093D01850883FC
:105B800017CD11166705119287AA0A4BC8A406AA59
:105B90001F3201468060127552FE1142F0D50DD2BF
:105BA00081610AAB741910422C760C99AEAE066670
:105BB000AF39092DAF39092DFC7D0A24418508F63E
:105BC000F9D5116EFB410803FB410803061C11E9DE
:105BD000061C11E971260866712608661ED705772E
:105BE0001ED70577DB620A0442C310FEEA650B008C
:105BF000D07902ECD07902ECF30A121884AA0815C5
:105C0000C45409EB295E1111BD9F101C6ADD0E1AE8
:105C1000DD3C0115067A06DA067A06DAB5CE12E21E
:105C2000931F0E5F740211C147730E772D67060430
:105C30002E5107CA6B4506B81CF7125FC59A11783A
:105C4000CF7E014ACF7E014A77D30D21D683107AC9
:105C50001A7110BD9743062BD2CD0ACEA41C06653F
:105C60001156136488A012F6C2080BEAC2080BEAA8
:105C7000C01B1195C01B1195F8580F5302E30C5926
:105C8000F7B30A5C5E59135A7F6212A02563315D37
:105C90002050726F6772616D20426C61636B2020CF
:105CA0002020202020325D2050726F6772616D20AD
:105CB0004379616E202020202020202020335D2089
:105CC00050726F6772616D204D6167656E746120FF
:105CD00020202025630D0A002563345D2050726F5B
:105CE0006772616D2059656C6C6F772020202020D1
:105CF00020355D2050726F6772616D204C2F4379A3
:105D0000616E20202020202020365D2050726F6799
:105D100072616D204C2F4D6167656E746120202586
:105D2000630D0A0025633D3D3D3D3D3D3D3D3D3D0F
:105D30003D3D3D3D3D3D3D3D3D3D3D3D3D3D3D3D93
:105D40003D3D3D3D3D3D3D3D3D3D3D3D3D3D3D3D83
:105D50003D3D3D3D3D3D3D3D3D3D3D3D3D3D3D3D73
:105D60003D3D3D3D3D3D3D3D3D3D3D25630D0A00F5
:105D70002563375D2050726F6772616D20436C65DB
:105D8000616E696E6720202020385D2050726F6739
:105D900072616D204D61696E74656E616E63652020
:105DA00020395D2050726F6772616D2044756D6D92
:105DB0007920202020202025630D0A002563415DE5
:105DC000205265616420454550524F4D20202020CF
:105DD0002020202020425D205265616420554944E6
:105DE00020286D756C74692D64726F7029435D2075
:105DF00053656C656374205365696B6F2F4F434522
:105E000020202025630D0A002563445D205365741E
:105E100020446576696365204461746520202020F4
:105E200020455D20436F7079204465766963652065
:105E3000496D61676520202020465D2050617374A4
:105E4000652044657669636520496D616765202535
:105E5000630D0A002563475D2050757263686173A6
:105E600065205265736574732020202020485D20D2
:105E70004368616E676520454550524F4D2064610F
:105E80007461202020495D20526561642055494499
:105E9000202873696E676C6529202025630D0A0030
:105EA00025634A5D20546F6767656C206F75747059
:105EB0007574207479706520204B5D2050726F6777
:105EC00072616D2053657269616C697A6572202018
:105ED000204C5D20467574757265205573652020D1
:105EE0002020202020202025630D0A00467574758F
:105EF000726520546563686E6F6C6F6769657300C7
:105F00002B3237283231293937362D3538313100A7
:105F1000202020202020207777772E6675747572D8
:105F200065746563686E6F6C6F676965732E636F08
:105F30002E7A61000D0A454550524F4D2070726F08
:105F40006772616D6D696E67206661696C65642159
:105F50000D0A000028506F737369626C65206361DD
:105F60007573653A204F545020626974206973201C
:105F7000736574206F7220736F20746865204545C7
:105F800050524F4D206E6565647320746F206265BA
:105F9000207265706C61636564290D0A00000D0A4A
:105FA000454550524F4D2070726F6772616D6D693B
:105FB0006E67206661696C6564210D0A00002854D3
:105FC000686520454550524F4D206661696C656497
:105FD00020746F2072657461696E207772697474C1
:105FE000656E20646174612E2020546865206465AC
:105FF00076696365206E6565647320746F206265E1
:10600000207265706C61636564290D0A0000437538
:106010007272656E7420646576696365206461746C
:10602000653A200025752F25752F254C753A2020BF
:10603000202052657065617420436F756E746572BF
:106040003A2D20254C750D0A00004465766963657C
:106050002053657269616C204E756D6265723A25D8
:106060006C75202D205265736574206C6F673A251E
:10607000750D0A0A000028506C65617365204E4F4B
:1060800054453A207468652061626F766520696EB8
:10609000666F726D6174696F6E206D7573742062C6
:1060A000652071756F746564207768656E20707502
:1060B0007263686173696E67206372656469747383
:1060C0002E0D0A005468697320696E666F726D61E7
:1060D00074696F6E206973207573656420746F2016
:1060E00067656E65726174652061206B65792074E7
:1060F0006861742077696C6C2062652073656E74CA
:10610000206261636B20746F20796F752E290D0AF0
:106110000A00437265646974732072656D61696E0B
:10612000696E673A20256C750D0A0A000D0A456EE6
:1061300074657220746865206E756D626572206F7B
:106140006620726573657420637265646974732078
:106150006265696E67207075726368617365643A21
:106160002D2020000D0A456E74657220746865202C
:10617000343020636861726163746572206B657985
:10618000636F646520737570706C696564206279F3
:1061900020003A2D200D0A000D0A52657365742007
:1061A0006372656469747320616D6D656E646564A6
:1061B000207375636365737366756C6C79206672A2
:1061C0006F6D20256C7520746F20256C752E000076
:1061D0000D0A496E76616C696420636F64652E00F8
:1061E0002A2A2A2A00005220452053204520540004
:1061F0005720522049205420452020202050205252
:10620000204F2043204520532053000020202053BE
:106210002055204320432045205320462055204C24
:106220002A2A2A2A00000A0A0D524553455420639F
:106230006F756E7465722069732061646A7573741A
:10624000656420746F3A20256C750A0D00000D0AF4
:1062500020284E6F20637265646974732072656DC7
:1062600061696E696E672E2050757263686173652F
:1062700020637265646974732066726F6D20465482
:106280002E290D0A000043415554494F4E212059F3
:106290006F75206F6E6C79206861766520256C754E
:1062A00020637265646974002072656D61696E694E
:1062B0006E672E2050757263686173652063726526
:1062C000646974732066726F6D200D0A000020628D
:1062D00065666F726520796F757220637265646997
:1062E000747320636F756E74657220726561636884
:1062F0006573207A65726F2E0000202020202020F8
:10630000000020202020256300002020202025637D
:10631000204D61696E204D656E75202D2053656995
:106320006B6F204920496E666F746563682028454D
:106330005529204368697020526570726F677261D9
:106340006D6D6572202020256300202020202563AC
:10635000204D61696E204D656E75202D2053656955
:106360006B6F204920496E666F7465636820284111
:1063700073696129204368697020526570726F6784
:1063800072616D6D657220256300202020202563D9
:10639000204D61696E204D656E75202D204F43455F
:1063A00020437320363036302043686970205265B0
:1063B00070726F6772616D6D6572202020202020E1
:1063C000202020202020202563002020202025635D
:1063D000204D61696E204D656E75202D202A2A2A78
:1063E000204E6F204F454D2073656C656374656466
:1063F000202A2A2A204368697020526570726F67CC
:1064000072616D6D6572202563000D0A46616D69CC
:106410006C7920436F64653A202532582020494426
:106420003A200000204352433A20253258000D0AFA
:10643000204E6F2064657669636573206F6E2074EB
:10644000686520312D5769726520627573000D0AE9
:106450004465766963652F732070726573656E7429
:106460002C20627574206E6F7420746865206D75C1
:106470006C74692D64726F702076617269657479CD
:1064800000000A0D454550524F4D20636865636B0F
:1064900073756D20636F6D7075746564202D202594
:1064A0003258253258202000454550524F4D20701B
:1064B000726F6772616D206661696C656421202866
:1064C0004F5450206269742070726F6261626C79FF
:1064D0002073657429005741524E494E473A205463
:1064E00068652055494420646964206E6F7420708B
:1064F000726F6772616D2073756363657373667520
:106500006C6C792E2050726F6772616D20616761CB
:10651000696E00000D0A54686520454550524F4D84
:106520002064657669636520636F756C64206E6FA7
:106530007420626520696E697469616C697A65644A
:106540002E2052657475726E206368697020746FB6
:106550002046542E0000454550524F4D204D656D4C
:106560006F72792064756D70202D2036342078206C
:10657000313662697420576F726473203D20314B4D
:10658000620D0A000D0A0A43686970204461746153
:1065900000000D0A3D3D3D3D3D3D3D3D3D000D0AA8
:1065A000436F6C6F75723A200000426C61636B0040
:1065B0004379616E00004D6167656E7461005965D5
:1065C0006C6C6F7700004C69676874204379616E6A
:1065D00000004C69676874204D6167656E746100E6
:1065E000436C65616E696E6700004D61696E74652C
:1065F0006E616E63650044756D6D7900496E7661FC
:106600006C696420436F6C6F757220446566696EB7
:106610006974696F6E000D0A4F454D204272616EBC
:10662000643A20005365696B6F205336342F313044
:10663000302000004F434520494A43363130200086
:106640004850393030302F313030303020004E6FEC
:10665000742064657465726D696E61626C650000BA
:106660000D0A4E6F74653A205468652055494420E0
:10667000646576696365206F6E2074686520636861
:106680006970206973206E6F742066756E6374691B
:106690006F6E696E6721212100002D2062757420C4
:1066A00063616E6E6F742062652070726F677261D5
:1066B0006D6D6564207769746820746869732072F1
:1066C000657365747465722E000043757272656E31
:1066D0007420696E6B206C6576656C3A28556E6423
:1066E000657220636F6E737472756374696F6E2167
:1066F000290D0A0050726F74656374696F6E2052C1
:1067000065676973746572205374617475733A2098
:10671000454550524F4D206C6F636B2069732000CC
:106720006E6F74206163746976617465642E000015
:10673000616374697661746564202D207265706C84
:1067400061636520454550524F4D2E000D0A436848
:1067500065636B73756D207374617475733A200093
:10676000556E7375636365737366756C6C792063BE
:1067700068616E67656420746F2025325825325831
:106780002E000D0A436F7272656374656420746F26
:10679000202532582532580D0A004E6F20636F7243
:1067A00072656374696F6E20706572666F726D6575
:1067B000642E20436865636B73756D206973206375
:1067C0006F72726563742E0D0A00496E70757420C5
:1067D0006164647265737320746F20777269746585
:1067E00020746F3A2D2000000A0D496E70757420D8
:1067F0006461746120776F726420746F20777269AE
:1068000074653A2D00000A0A0D454550524F4D203F
:106810007772697474656E3A20416464726573734B
:106820003A2D000030332C303520262030442044CF
:106830006174613A2D2532582532580030422026A5
:1068400020323020446174613A2D25325825325867
:1068500000003046202620323320446174613A2DF6
:10686000253258253258000031312026203234207C
:10687000446174613A2D2532582532580000304663
:10688000202620323320446174613A2D2532582568
:106890003258000025325820446174613A2D253267
:1068A00058253258000043757272656E7420726507
:1068B000736574206372656469747320636F756EA9
:1068C0007465723A20256C750A0D00000D0A496E38
:1068D00070757420646576696365207965617228D6
:1068E0003230303720746872752032303137293AAF
:1068F00020000D0A496E70757420646576696365C1
:10690000206D6F6E74682831207468727520313282
:1069100029203A2000000D0A496E707574206465C4
:106920007669636520646179283120746872752006
:10693000333129203A2000000D0A44617465206338
:1069400068616E6765207375636365737366756CE4
:106950006C2E0D0A000050726F6772616D6D656478
:106960002063686970732077696C6C206E6F772084
:10697000636F6E7461696E207468697320656E63FD
:106980006F64656420646174652076616C75652E42
:10699000202532582532580D0A000D0A532E2E5349
:1069A00065696B6F2845552920412E2E5365696B0B
:1069B0006F284173696129204F2E2E4F43452000D7
:1069C0000D0A496E736572742061206368697020D6
:1069D000616E6420707265737320616E79206B65DF
:1069E0007920746F20636F6E74696E75652E2E2E1C
:1069F00000000D0A53686F756C642074686520642C
:106A000061746120626520636C65617265642074E5
:106A10006F2074686174206F662061206E65772036
:106A2000636869703F28592F4E292E2E2E000D0ABB
:106A30004E6F7720636F7079696E67206368697045
:106A4000206461746120746F20696D6167652E2018
:106A500000000D0A5768617420636F6C6F757220B7
:106A600073686F756C642074686520636869702052
:106A700062652070726F6772616D6D656420696E0A
:106A8000746F3F0D0A00313D426C61636B2C323DE7
:106A90004379616E2C333D4D6167656E74612C34B2
:106AA0003D59656C6C6F772C353D4C696768745F38
:106AB0004379616E2C363D4C696768745F4D616740
:106AC000656E746120000D0A436F6D706C657465AE
:106AD000640D0A000D0A496E7365727420612046C8
:106AE00054206368697020696E7420746865207032
:106AF000726F6772616D6D657220616E6420707275
:106B000065737320616E79206B657920746F2063E3
:106B10006F6E74696E75652E2E2E00000D0A506121
:106B20007374696E672074686520696D616765209C
:106B3000746F2074686520636869702E2000202AB5
:106B40002A2A205320452049204B204F2020532023
:106B5000362034202D204361727472696467652089
:106B60004368697020526573657474657220566558
:106B70007220312E34352D313120436F7079726996
:106B800067687428432932303131202A2A2A0D0AB5
:106B90000000202020202020202020200000202D68
:106BA0002054656C3A002020202020202020202026
:106BB0002020202000000D0A53656C656374206F4F
:106BC0007074696F6E3A2020000020466F726D610C
:106BD00074206973204E6F726D616C0A0D0020463F
:106BE0006F726D61742069732073657420666F72B3
:106BF0002046696C652044756D70696E670A0D00EA
:106C0000496E76616C6964204D656E752053656CC4
:106C1000656374696F6E0A0D00000D0A0A2E2E2E30
:106C20002E2E707265737320616E79206B657920EA
:106C3000746F20636F6E74696E75652E0000939299
:106C40008A9293948A94938693988A98939A8A9A2C
:106C5000939C8A8CC1EF5DF092908990000CEA6A57
:106C6000ED0EE96EEF5011E0060E016EBF0E006EE4
:106C70000400002EFDD7012EF9D77A0E006E002EEB
:106C8000FED700D00400EF2EEFD7000C9280000C4E
:106C90001B0E04009EA8FDD7AD6E5B0E04009EA8DF
:106CA000FDD7AD6E320E04009EA8FDD7AD6E4A0E24
:106CB00004009EA8FDD7AD6E000C0900F5520EE051
:106CC000F6CFF2F0F7CFF3F0F55004009EA8FDD711
:106CD000AD6EF2C0F6FFF3C0F7FFEFD7000CF55131
:106CE000016AF45D03E2F4C000F00CD0006A080E03
:106CF000F66FF4370036F551005CD8B0006E0136FF
:106D0000F62FF7D7000C0150F2C0F4F0640EF56FC7
:106D1000E6DF00C0F2F00150300E07E1F3A30ED021
:106D2000F3B70CD0F3B9200E03D0F397F399F381A6
:106D30000126015004009EA8FDD7AD6EF2C0F4F00C
:106D40000A0EF56FCCDF00C0F2F00150300E06E104
:106D5000F3B70AD0F3A108D0F3B9200E01260150F1
:106D600004009EA8FDD7AD6E300EF227F25104004C
:106D70009EA8FDD7AD6E000CEACFFAF0E9CFF9F08E
:106D8000F339F009F56FF527E20FF66F320FF86F60
:106D9000F3510F0BF627F627F827E90FF76FF727C0
:106DA000F727F2390F0BF727F827F737F837F81FCF
:106DB000F837F2510F0BF827F537070EF46F0A0E6C
:106DC000F707F827FDE3F607F727FDE3F507F627B2
:106DD000FDE3F407F527FDE3EA6AF40EE96E070E1A
:106DE000F915F99DE926F80EE95CD8B4F98DEF5054
:106DF000006E08E1F9BD06D0F9B90DD0F9B702D09F
:106E0000200E03D0F987F999300E002600500400B7
:106E10009EA8FDD7AD6EEE50F9ADE5D7000C090088
:106E2000F6CFF3F0F7CFF4F0F55004009EA8FDD7AD
:106E3000AD6EF3C0F6FFF4C0F7FFF22FF0D7000CF1
:106E4000EB511F0BEE6FEC31F36FEB31F26FF3335D
:106E5000F233F333F233F333F233F333F233070E17
:106E6000F317F2510F0BEF6FD890F36BEC31F26F19
:106E7000D00EF225F06F070EF321F16F0E0EF66EB5
:106E8000600EF76E1ADFED5334E0EEC0F2F01B0E29
:106E9000F36F39DF2F0E04009EA8FDD7AD6EEFC053
:106EA000F2F01B0EF36F2FDF2F0E04009EA8FDD70C
:106EB000AD6E100EE96EF1C0F3F0F0C0F2F05CDFE1
:106EC0002D0EF66E600EF76E160EF26FA8DF100E26
:106ED000E96E45C0F3F044C0F2F04EDF0D0E040041
:106EE0009EA8FDD7AD6E0A0E04009EA8FDD7AD6E1C
:106EF00025D0EEC0F2F01B0EF36F05DF2F0E04005D
:106F00009EA8FDD7AD6EEFC0F2F01B0EF36FFBDE57
:106F10002F0E04009EA8FDD7AD6E100EE96EF1C0D5
:106F2000F3F0F0C0F2F028DF0D0E04009EA8FDD7AC
:106F3000AD6E0A0E04009EA8FDD7AD6E000CFA0ED1
:106F4000F66E620EF76EB9DEF2CF66F0F29EAA6AB6
:106F5000130EA96EA69CA69EA680A85066BEF28EB1
:106F6000676EF2CF68F0F29EAA6A140EA96EA69C14
:106F7000A69EA680A85068BEF28E696E67C06BF0B0
:106F800069C06AF06BC0ECF06AC0EBF0010EED6F07
:106F900057DF0A0E04009EA8FDD7AD6E020EF66EF6
:106FA000630EF76E040EF26F3ADFC90E04009EA85E
:106FB000FDD7AD6E656A6550360807E3CD0E040057
:106FC0009EA8FDD7AD6E652AF6D7BB0E04009EA81D
:106FD000FDD7AD6E0D0E04009EA8FDD7AD6E0A0E56
:106FE00004009EA8FDD7AD6E475005E0010A1CE0E5
:106FF000030A33E04BD00A0EF66E630EF76E040EF2
:10700000F26F0DDFBA0E04009EA8FDD7AD6E100E14
:10701000F66E630EF76E370EF26F01DFBA0E0400E4
:107020009EA8FDD7AD6E4AD04A0EF66E630EF76E7F
:10703000040EF26FF4DEBA0E04009EA8FDD7AD6E0A
:10704000500EF66E630EF76E370EF26FE8DEBA0E74
:1070500004009EA8FDD7AD6E31D08A0EF66E630E89
:10706000F76E040EF26FDBDEBA0E04009EA8FDD7A9
:10707000AD6E900EF66E630EF76E370EF26FCFDECA
:10708000BA0E04009EA8FDD7AD6E18D0CA0EF66EDB
:10709000630EF76E040EF26FC2DEBA0E04009EA8F5
:1070A000FDD7AD6ED00EF66E630EF76E370EF26F33
:1070B000B6DEBA0E04009EA8FDD7AD6E0D0E04001C
:1070C0009EA8FDD7AD6E0A0E04009EA8FDD7AD6E3A
:1070D000DA0E04009EA8FDD7AD6EC40E04009EA873
:1070E000FDD7AD6EC40E04009EA8FDD7AD6EC40ED4
:1070F00004009EA8FDD7AD6ED00E04009EA8FDD75B
:10710000AD6E656A6550360807E3C40E04009EA89C
:10711000FDD7AD6E652AF6D7D00E04009EA8FDD728
:10712000AD6E656A6550080807E3C40E04009EA8AA
:10713000FDD7AD6E652AF6D7BF0E04009EA8FDD719
:10714000AD6E0D0E04009EA8FDD7AD6E0A0E0400B4
:107150009EA8FDD7AD6EB30E04009EA8FDD7AD6E00
:107160008E0EF66E5C0EF76E450EF26F58DEB30EA5
:1071700004009EA8FDD7AD6E0D0E04009EA8FDD79D
:10718000AD6E0A0E04009EA8FDD7AD6EB30E0400CE
:107190009EA8FDD7AD6EDA0EF66E5C0EF76E450E4C
:1071A000F26F3DDEB30E04009EA8FDD7AD6E0D0E4E
:1071B00004009EA8FDD7AD6E0A0E04009EA8FDD760
:1071C000AD6EB30E04009EA8FDD7AD6E260EF66E12
:1071D0005D0EF76E450EF26F22DEB30E04009EA820
:1071E000FDD7AD6E0D0E04009EA8FDD7AD6E0A0E44
:1071F00004009EA8FDD7AD6EB30E04009EA8FDD777
:10720000AD6E720EF66E5D0EF76E450EF26F07DE16
:10721000B30E04009EA8FDD7AD6E0D0E04009EA80F
:10722000FDD7AD6E0A0E04009EA8FDD7AD6EB30E5D
:1072300004009EA8FDD7AD6E260EF66E5D0EF76EAD
:10724000450EF26FECDDB30E04009EA8FDD7AD6EC7
:107250000D0E04009EA8FDD7AD6E0A0E04009EA878
:10726000FDD7AD6EB30E04009EA8FDD7AD6EBE0E69
:10727000F66E5D0EF76E450EF26FD1DDB30E0400B3
:107280009EA8FDD7AD6E0D0E04009EA8FDD7AD6E75
:107290000A0E04009EA8FDD7AD6EB30E04009EA892
:1072A000FDD7AD6E0A0EF66E5E0EF76E450EF26FEE
:1072B000B6DDB30E04009EA8FDD7AD6E0D0E040022
:1072C0009EA8FDD7AD6E0A0E04009EA8FDD7AD6E38
:1072D000B30E04009EA8FDD7AD6E560EF66E5E0E80
:1072E000F76E450EF26F9BDDB30E04009EA8FDD72E
:1072F000AD6E0D0E04009EA8FDD7AD6E0A0E040003
:107300009EA8FDD7AD6EB30E04009EA8FDD7AD6E4E
:10731000A20EF66E5E0EF76E450EF26F80DDB30EB6
:1073200004009EA8FDD7AD6E0D0E04009EA8FDD7EB
:10733000AD6E0A0E04009EA8FDD7AD6EC00E04000F
:107340009EA8FDD7AD6E656A6550440807E3C40E7C
:1073500004009EA8FDD7AD6E652AF6D7D90E0400AD
:107360009EA8FDD7AD6E5DEF5EF0F26BF16BED3573
:10737000EE6FEE37FC0EEE17060EEF6F010EF06F9C
:10738000F051050805E3D890EE37EF37F02BF8D72A
:10739000939A8A8A010EF06FF051190819E3D89078
:1073A000EE37EF3702E28A9601D08A869396939859
:1073B0008A8893988A98F051090808E2938481B4E6
:1073C00002D0D89001D0D880F137F237F02BE4D733
:1073D000939A8A9AF1C001F0F2C002F0000CF2CF49
:1073E00071F0F29EAA6A100EA96EA69CA69EA680B7
:1073F000A85071BEF28E726EF2CF73F0F29EAA6A3E
:10740000110EA96EA69CA69EA680A85073BEF28EF1
:10741000746E72C06CF074C06BF06C50260837E26A
:10742000FF0A03E16B50100832E26C6A320E6B6E99
:107430006CC071F0726AAA6A100EA96E71C0A8FFC2
:10744000A69CA69EA684F250006EF29E0F01550ED9
:10745000A76EAA0EA76EA682A6B2FED7A69400506B
:10746000F212AA6A110EA96E6BC0A8FFA69CA69E76
:10747000A684F2CF00F0F29E550EA76EAA0EA76E5C
:10748000A682A6B2FED7A6940050F21200016B525B
:1074900013E16C5211E14E0EF66E620EF76E0DDCCA
:1074A000080E716EFA0EED6F2FEC36F0712EFAD7D2
:1074B000000E016E83D082D06C523CE16B503108DB
:1074C00039E3860EF66E620EF76E170EF26FA7DCCA
:1074D000100EE96E6CC0F3F06BC0F2F04DDCA00E44
:1074E000F66E620EF76E070EF26F99DC6C5203E1D6
:1074F0006B50010805E2730E04009EA8FDD7AD6E27
:10750000A80EF66E620EF76E5DEC36F0EC0EF66EBF
:107510005E0EF76E5DEC36F0CE0EF66E620EF76E16
:107520005DEC36F0080E716EFA0EED6F2FEC36F052
:10753000712EFAD7F2CF71F0F29EAA6A160EA96EDA
:10754000A69CA69EA680A85071BEF28E726EF2CF47
:1075500073F0F29EAA6A170EA96EA69CA69EA6803C
:10756000A85073BEF28E746EF2CF75F0F29EAA6AC6
:10757000180EA96EA69CA69EA680A85075BEF28E77
:10758000766E706A72C06FF074C06EF076C06DF087
:107590006D50DD0810E16E5026080DE16F520BE1D1
:1075A000705209E16C5207E16B501D0804E3000EB4
:1075B000016E04D003D0010E016E00D0000CF3392F
:1075C000F46FF437F437C00EF417040EF56F010EA4
:1075D000F66FF651050805E3D890F437F537F62B2A
:1075E000F8D7939C8A8C939A8A8A010EF66FF6518B
:1075F00009080EE3D890F437F53702E28A9601D0F5
:107600008A86939693988A8893988A98F62BEFD7D0
:1076100093968A96939C8A9C939A8A9A000C030E5E
:10762000F36FCDDF6BC06DF06CC06EF0100E6F6E3F
:10763000010E706E716A7150060807E3D8906D36BE
:107640006E366F367036712AF6D793928A92939C73
:107650008A8C939A8A8A010E716E7150190810E310
:10766000D8906D366E366F36703602E28A9601D04B
:107670008A86939693988A8893988A98712AEDD7E8
:1076800093968A96939C8A9C939A8A9A0400070EF2
:10769000006E002EFED700D0939A8A8A938481A42C
:1076A000FDD7939A8A9AF36B8ADF5BEF3BF0FF0E6C
:1076B0006C6E6B6EB4D7ED6B58DE02C06CF001C01F
:1076C0006BF0013C03D06C3C01D003D0000E016E86
:1076D00018D0216A0F0E206E420E236E400E226ECD
:1076E000296A286A2B6A2A6A336A326A376A366AD2
:1076F000FF0E3B6E3A6E3F6A3E6A416E406E010E6F
:10770000016E000C6C506E02F3CF01F0F4CF00F06C
:107710006F02F35000266D506E02F3500020026E8F
:10772000000CF2CF6CF0F29EAA6A300EA96EA69CF5
:10773000A69EA680A8506CBEF28E6D6EF2CF6EF043
:10774000F29EAA6A310EA96EA69CA69EA680A8509B
:107750006EBEF28E6F6E6DC06BF06FC06AF06950D6
:10776000F70F29E2090F85EF3DF0156A146A23D05F
:10777000100E156E146A1FD0200E156E146A1BD0E1
:10778000300E156E146A17D0400E156E146A13D0A1
:10779000500E156E146A0FD0F00E156E040E146E96
:1077A0000AD0F00E156E050E146E05D0F00E156E93
:1077B000060E146E00D0110E176E166A6A346C6EC7
:1077C0006B346D6E6C366D36FC0E6C166DC003F04E
:1077D0006C506DC0F7FF7BEC1BF0056E6A346C6E6D
:1077E0006B346D6E6C366D36FC0E6C16010E6C24AF
:1077F000016E000E6D20036E015003C0F7FF7BEC9D
:107800001BF0066E6A346C6E6B346D6E6C366D36C2
:10781000FC0E6C16020E6C24016E000E6D20036EC1
:10782000015003C0F7FF7BEC1BF0076E6A346C6EEF
:107830006B346D6E6C366D36FC0E6C16030E6C245C
:10784000016E000E6D20036E015003C0F7FF7BEC4C
:107850001BF00B6E6BC06DF06AC06CF06F6A140E9B
:107860006E6E50DF02C06DF001C06CF002C003F01C
:10787000015002C0F7FF04EC04F00900F5CF03F05B
:10788000186E03C019F06BC06DF06AC06CF06F6ABF
:10789000140E6E6E37DF02C06DF001C06CF0020E88
:1078A0000124016E000E0220036E015003C0F7FF99
:1078B00004EC04F00900F5CF03F01C6E03C01DF0CA
:1078C0006BC06DF06AC06CF06F6A140E6E6E1ADFDA
:1078D00002C06DF001C06CF0040E0124016E000EB8
:1078E0000220036E015003C0F7FF04EC04F009000E
:1078F000F5CF03F0246E03C025F06BC06DF06AC0B5
:107900006CF06F6A140E6E6EFDDE02C06DF001C089
:107910006CF0060E0124016E000E0220036E015071
:1079200003C0F7FF04EC04F00900F5CF03F0266E66
:1079300003C027F06BC06DF06AC06CF06F6A140E64
:107940006E6EE0DE02C06DF001C06CF0080E012426
:10795000016E000E0220036E015003C0F7FF04EC1D
:1079600004F00900F5CF03F02C6E03C02DF06BC0BE
:107970006DF06AC06CF06F6A140E6E6EC3DE02C0EA
:107980006DF001C06CF00A0E0124016E000E0220A1
:10799000036E015003C0F7FF04EC04F00900F5CFBB
:1079A00003F0306E03C031F06BC06DF06AC06CF054
:1079B0006F6A140E6E6EA6DE02C06DF001C06CF030
:1079C0000C0E0124016E000E0220036E015003C054
:1079D000F7FF04EC04F00900F5CF03F0346E03C0A8
:1079E00035F06BC06DF06AC06CF06F6A140E6E6E8D
:1079F00089DE02C06DF001C06CF00E0E0124016E34
:107A0000000E0220036E015003C0F7FF04EC04F0E7
:107A10000900F5CF03F0386E03C039F06BC06DF08C
:107A20006AC06CF06F6A140E6E6E6CDE02C06DF090
:107A300001C06CF0100E0124016E000E0220036ED6
:107A4000015003C0F7FF04EC04F00900F5CF03F088
:107A50003C6E03C03DF06BC06DF06AC06CF06F6AA5
:107A6000140E6E6E4FDE02C06DF001C06CF0120E8F
:107A70000124016E000E0220036E015003C0F7FFC7
:107A800004EC04F00900F5CF03F0426E03C043F0AC
:107A90006A2AD8B46B2A6B50010807E2FF0A03E197
:107AA0006A50580802E26B6A6A6A6BC06CF06D6AD1
:107AB000AA6A300EA96E6CC0A8FFA69CA69EA684DA
:107AC000F250006EF29E0F01550EA76EAA0EA76E21
:107AD000A682A6B2FED7A6940050F212AA6A310E70
:107AE000A96E6AC0A8FFA69CA69EA684F2CF00F04D
:107AF000F29E550EA76EAA0EA76EA682A6B2FED75C
:107B0000A6940050F2120001000CE824F76AF73640
:107B1000250FF66E7B0EF7220A00F550FA6E08006C
:107B2000F550F96E6A7770777877807788779077F5
:107B30009877A277AC77F2CF6CF0F29EAA6A320EF9
:107B4000A96EA69CA69EA680A8506CBEF28E6D6EF5
:107B5000F2CF6EF0F29EAA6A330EA96EA69CA69E84
:107B6000A680A8506EBEF28E6F6E6DC06BF06FC0B7
:107B70006AF06950F70F29E2090F8CEF3FF0156AA0
:107B8000146A23D0100E156E146A1FD0200E156EC5
:107B9000146A1BD0300E156E146A17D0400E156E85
:107BA000146A13D0500E156E146A0FD0F00E156EB5
:107BB000040E146E0AD0F00E156E050E146E05D06C
:107BC000F00E156E060E146E00D0110E176E166AAA
:107BD0006A346C6E6B346D6E6C366D36FC0E6C16E2
:107BE0006DC003F06C506DC0F7FF0DEC24F0056E16
:107BF0006A346C6E6B346D6E6C366D36FC0E6C16C2
:107C0000010E6C24016E000E6D20036E015003C046
:107C1000F7FF0DEC24F0066E6A346C6E6B346D6EFB
:107C20006C366D36FC0E6C16020E6C24016E000E66
:107C30006D20036E015003C0F7FF0DEC24F0076EBA
:107C40006A346C6E6B346D6E6C366D36FC0E6C1671
:107C5000030E6C24016E000E6D20036E015003C0F4
:107C6000F7FF0DEC24F00B6E6BC06DF06AC06CF08A
:107C70006F6A140E6E6E46DD02C06DF001C06CF0CE
:107C800002C003F0015002C0F7FF32EC20F00900FF
:107C9000F5CF03F0186E03C019F06BC06DF06AC029
:107CA0006CF06F6A140E6E6E2DDD02C06DF001C0B7
:107CB0006CF0020E0124016E000E0220036E0150D2
:107CC00003C0F7FF32EC20F00900F5CF03F01C6E83
:107CD00003C01DF06BC06DF06AC06CF06F6A140ECB
:107CE0006E6E10DD02C06DF001C06CF0040E012458
:107CF000016E000E0220036E015003C0F7FF32EC4C
:107D000020F00900F5CF03F0246E03C025F06BC00E
:107D10006DF06AC06CF06F6A140E6E6EF3DC02C018
:107D20006DF001C06CF0060E0124016E000E022001
:107D3000036E015003C0F7FF32EC20F00900F5CFCD
:107D400003F0266E03C027F06BC06DF06AC06CF0C4
:107D50006F6A140E6E6ED6DC02C06DF001C06CF05E
:107D6000080E0124016E000E0220036E015003C0B4
:107D7000F7FF32EC20F00900F5CF03F02C6E03C0C2
:107D80002DF06BC06DF06AC06CF06F6A140E6E6EF1
:107D9000B9DC02C06DF001C06CF00A0E0124016E66
:107DA000000E0220036E015003C0F7FF32EC20F0FA
:107DB0000900F5CF03F0306E03C031F06BC06DF0F9
:107DC0006AC06CF06F6A140E6E6E9CDC02C06DF0BF
:107DD00001C06CF00C0E0124016E000E0220036E37
:107DE000015003C0F7FF32EC20F00900F5CF03F09B
:107DF000346E03C035F06BC06DF06AC06CF06F6A12
:107E0000140E6E6E7FDC02C06DF001C06CF00E0EC1
:107E10000124016E000E0220036E015003C0F7FF23
:107E200032EC20F00900F5CF03F0386E03C039F0D2
:107E30006BC06DF06AC06CF06F6A140E6E6E62DC1F
:107E400002C06DF001C06CF0100E0124016E000E36
:107E50000220036E015003C0F7FF32EC20F009004E
:107E6000F5CF03F03C6E03C03DF06BC06DF06AC00F
:107E70006CF06F6A140E6E6E45DC02C06DF001C0CE
:107E80006CF0120E0124016E000E0220036E0150F0
:107E900003C0F7FF32EC20F00900F5CF03F0426E8B
:107EA00003C043F06A2AD8B46B2A6B5203E16A50CC
:107EB000620802E26B6A6A6A6BC06CF06D6AAA6A59
:107EC000320EA96E6CC0A8FFA69CA69EA684F25096
:107ED000006EF29E0F01550EA76EAA0EA76EA68227
:107EE000A6B2FED7A6940050F212AA6A330EA96E6B
:107EF0006AC0A8FFA69CA69EA684F2CF00F0F29EC0
:107F0000550EA76EAA0EA76EA682A6B2FED7A6949D
:107F10000050F2120001000CE824F76AF736330F24
:107F2000F66E7F0EF7220A00F550FA6E0800F55043
:107F3000F96E7E7B847B8C7B947B9C7BA47BAC7B6F
:107F4000B67BC07BF2CF6CF0F29EAA6A340EA96EAB
:107F5000A69CA69EA680A8506CBEF28E6D6EF2CF37
:107F60006EF0F29EAA6A350EA96EA69CA69EA68009
:107F7000A8506EBEF28E6F6E6DC06BF06FC06AF06F
:107F80006950F70F29E2090F9EEF41F0156A146A54
:107F900023D0100E156E146A1FD0200E156E146AB1
:107FA0001BD0300E156E146A17D0400E156E146A71
:107FB00013D0500E156E146A0FD0F00E156E040E0D
:107FC000146E0AD0F00E156E050E146E05D0F00E6C
:107FD000156E060E146E00D0110E176E010E166E81
:107FE0006A346C6E6B346D6E6C366D36FC0E6C16CE
:107FF0006DC003F06C506DC0F7FFAFEC2CF0056E58
:108000006A346C6E6B346D6E6C366D36FC0E6C16AD
:10801000010E6C24016E000E6D20036E015003C032
:10802000F7FFAFEC2CF0066E6A346C6E6B346D6E3D
:108030006C366D36FC0E6C16020E6C24016E000E52
:108040006D20036E015003C0F7FFAFEC2CF0076EFC
:108050006A346C6E6B346D6E6C366D36FC0E6C165D
:10806000030E6C24016E000E6D20036E015003C0E0
:10807000F7FFAFEC2CF00B6E6BC06DF06AC06CF0CC
:108080006F6A140E6E6E82EC3BF002C06DF001C0A0
:108090006CF002C003F0015002C0F7FFD8EC24F0EE
:1080A0000900F5CF03F0186E03C019F06BC06DF036
:1080B0006AC06CF06F6A140E6E6E82EC3BF002C008
:1080C0006DF001C06CF0020E0124016E000E022062
:1080D000036E015003C0F7FFD8EC24F00900F5CF80
:1080E00003F01C6E03C01DF06BC06DF06AC06CF035
:1080F0006F6A140E6E6E82EC3BF002C06DF001C030
:108100006CF0040E0124016E000E0220036E01507B
:1081100003C0F7FFD8EC24F00900F5CF03F0246E7C
:1081200003C025F06BC06DF06AC06CF06F6A140E6E
:108130006E6E82EC3BF002C06DF001C06CF0060E7A
:108140000124016E000E0220036E015003C0F7FFF0
:10815000D8EC24F00900F5CF03F0266E03C027F019
:108160006BC06DF06AC06CF06F6A140E6E6E82ECBC
:108170003BF002C06DF001C06CF0080E0124016EEE
:10818000000E0220036E015003C0F7FFD8EC24F06C
:108190000900F5CF03F02C6E03C02DF06BC06DF01D
:1081A0006AC06CF06F6A140E6E6E82EC3BF002C017
:1081B0006DF001C06CF00A0E0124016E000E022069
:1081C000036E015003C0F7FFD8EC24F00900F5CF8F
:1081D00003F0306E03C031F06BC06DF06AC06CF01C
:1081E0006F6A140E6E6E82EC3BF002C06DF001C03F
:1081F0006CF00C0E0124016E000E0220036E015083
:1082000003C0F7FFD8EC24F00900F5CF03F0346E7B
:1082100003C035F06BC06DF06AC06CF06F6A140E6D
:108220006E6E82EC3BF002C06DF001C06CF00E0E81
:108230000124016E000E0220036E015003C0F7FFFF
:10824000D8EC24F00900F5CF03F0386E03C039F004
:108250006BC06DF06AC06CF06F6A140E6E6E82ECCB
:108260003BF002C06DF001C06CF0100E0124016EF5
:10827000000E0220036E015003C0F7FFD8EC24F07B
:108280000900F5CF03F03C6E03C03DF06BC06DF00C
:108290006AC06CF06F6A140E6E6E82EC3BF002C026
:1082A0006DF001C06CF0120E0124016E000E022070
:1082B000036E015003C0F7FFD8EC24F00900F5CF9E
:1082C00003F0426E03C043F06A2AD8B46B2A6B52A3
:1082D00003E16A50C80802E26B6A6A6A6BC06CF01C
:1082E0006D6AAA6A340EA96E6CC0A8FFA69CA69EF1
:1082F000A684F250006EF29E0F01550EA76EAA0ED4
:10830000A76EA682A6B2FED7A6940050F212AA6A61
:10831000350EA96E6AC0A8FFA69CA69EA684F2CFC1
:1083200000F0F29E550EA76EAA0EA76EA682A6B208
:10833000FED7A6940050F2120001000CE824F76A60
:10834000F736570FF66E830EF7220A00F550FA6ED5
:108350000800F550F96E8C7F927F9A7FA27FAA7FEA
:10836000B27FBA7FC47FCE7F030EF36FDFEC3AF0AB
:10837000ECC0EEF0EDC0EFF0EB514009F06F010EF4
:10838000F16FF26BF251060807E3D890EE37EF3742
:10839000F037F137F22BF6D7939C8A8C939A8A8A1E
:1083A000010EF26FF251190810E3D890EE37EF3753
:1083B000F037F13702E28A9601D08A869396939835
:1083C0008A8893988A98F22BEDD793968A96939CF5
:1083D0008A9C939A8A9A0400070E006E002EFED79C
:1083E00000D0939A8A8A938481A4FDD7939A8A9A1B
:1083F000F36BDFEC3AF0000C030EEB6F78C0EDF09E
:1084000077C0ECF0B1DF050EEB6F78C0EDF077C010
:10841000ECF0AADF0D0EEB6F78C0EDF077C0ECF05A
:10842000A3DF000CF0BF11D00F0E006EEF39001665
:108430000A0E005C03E2300E002602D0F051002646
:10844000005004009EA8FDD7AD6E0F0EEF170A0E68
:10845000EF5D02E2300E02D0F09FF051EF27EF51B6
:1084600004009EA8FDD7AD6E000C756A746A716A2F
:10847000715017080EE371C0EDF0B5EC39F002C091
:1084800073F001C072F07250742673507522712A15
:10849000EFD73E0EED6FB5EC39F002C077F001C0BA
:1084A00076F0013C03D0773C01D007D03E0EEB6F55
:1084B00075C0EDF074C0ECF057DF3F0EEB6F75C088
:1084C000EDF074C0ECF050DF75C076F0776A820E84
:1084D000F66E640EF76E1D0EF26F0FEC37F076C07D
:1084E000EFF0370EF06F9EDF74C0EFF0370EF06FD5
:1084F00099DF200E04009EA8FDD7AD6E200E04006B
:108500009EA8FDD7AD6EFAEF44F0030EEF5F0AE3CD
:10851000EA6AEF0EE96EEF5005E002D000000400B9
:10852000EF2EFCD7000C93908A900400030EEE6FA0
:10853000A20EEF6FEADFEE2FFBD793800400070E49
:10854000006E002EFED700D0938081B003D0000EC5
:10855000016E17D004006B0E006E002EFED700D007
:108560009380ED9181A0ED810400EF0EEF6FCDDFE0
:10857000EDA104D0010E016E04D003D0000E016EF7
:1085800000D0000C010EEE6FEE51080833E393901B
:108590008A90040000D000D0D890ED330EE3939081
:1085A0008A800400180E006E002EFED7000081B0F5
:1085B00003D0000E016E20D00DD093908A9004005D
:1085C000180E006E002EFED7000081A003D0000E12
:1085D000016E12D00400450E006E002EFED7000082
:1085E00093908A8004006D0E006E002EFED700006E
:1085F000EE2BCAD7010E016E000C010EEF6FEF518A
:1086000008081BE393908A90040000D000D0938068
:108610000400180E006E002EFED70000938081B07B
:1086200002D0D89001D0D880F0330400B60E006E8E
:10863000002EFED700D0EF2BE2D7F0C001F0000CE7
:1086400048B03DD00A0EF66E640EF76E0F0EF26F54
:108650000FEC37F004C0EFF0370EF06FE3DE1C0EC6
:10866000F66E640EF76E060EF26F0FEC37F0010E29
:10867000ED6FED51060815E3036AED51040FE96E45
:10868000000E0320EA6EEFCFEEF0EEC0EFF0370EF3
:10869000F06FC8DE200E04009EA8FDD7AD6EED2B56
:1086A000E8D7240EF66E640EF76E060EF26F0FEC2E
:1086B00037F00BC0EFF0370EF06FB4DE23D00D0EA5
:1086C00004009EA8FDD7AD6E0A0E04009EA8FDD73B
:1086D000AD6EED6BED51070815E3036AED51040F24
:1086E000E96E000E0320EA6EEFCFEEF0EEC0EFF081
:1086F000370EF06F97DE200E04009EA8FDD7AD6EFA
:10870000ED2BE8D7000CD76AD66AF2940CDF015241
:10871000FDE0F2A403D0000E016E38D0020EED6F22
:108720002FEC36F00400DD0EEF6FEFDE330EED6F51
:1087300029DFEC6BEC51070818E30400A60E006E6D
:10874000002EFED7036AEC51040F016E000E0322C7
:1087500001C0EDF003C0EEF050DFEEC0EAFFEDC067
:10876000E9FF01C0EFFFEC2BE5D7EB530DE068DF2D
:1087700048B00AD00A0E04009EA8FDD7AD6E0D0EBB
:1087800004009EA8FDD7AD6E010E016E000C756A47
:10879000746A735202E048EC36F0F2CF76F0F29E43
:1087A000AA6A100EA96EA69CA69EA680A85076BEA8
:1087B000F28E776EF2CF78F0F29EAA6A110EA96E51
:1087C000A69CA69EA680A85078BEF28E796E77C031
:1087D00075F079C074F07550260837E2FF0A03E19E
:1087E0007450100832E2756A320E746E75C076F0FD
:1087F000776AAA6A100EA96E76C0A8FFA69CA69EEC
:10880000A684F250006EF29E0F01550EA76EAA0EBE
:10881000A76EA682A6B2FED7A6940050F212AA6A4C
:10882000110EA96E74C0A8FFA69CA69EA684F2CFC6
:1088300000F0F29E550EA76EAA0EA76EA682A6B2F3
:10884000FED7A6940050F21200017150745E000E23
:10885000755A75C076F0776AAA6A100EA96E76C04E
:10886000A8FFA69CA69EA684F250006EF29E0F0161
:10887000550EA76EAA0EA76EA682A6B2FED7A69424
:108880000050F212AA6A110EA96E74C0A8FFA69C2D
:10889000A69EA684F2CF00F0F29E550EA76EAA0EF9
:1088A000A76EA682A6B2FED7A6940050F212E00EE2
:1088B000F66E610EF76E00015DEC36F0725207E164
:1088C000E60EF66E610EF76E5DEC36F006D0F00E39
:1088D000F66E610EF76E5DEC36F00C0EF66E620E03
:1088E000F76E5DEC36F0260EF66E620EF76E210E18
:1088F000F26F0FEC37F0100EE96E75C0F3F074C034
:10890000F2F0BCEC36F00A0E04009EA8FDD7AD6E66
:108910000D0E04009EA8FDD7AD6E080E766EFA0E01
:10892000ED6F2FEC36F0762EFAD7000C6E806D6A64
:108930006D50170830E3D8906D34036A140FE96E58
:10894000000E0320EA6EECCF72F0ED52EFCF71F023
:108950006DC0EBF072C0EDF071C0ECF005DD6DC0E4
:10896000EDF0B5EC39F002C070F001C06FF0D890B6
:108970006D34036A140FE96E000E0320EA6EECCF2B
:1089800003F0ED52EF506F5C03E10350705C01E0C7
:108990006E906D2ACDD76EB007D0A80EF66E640E1D
:1089A000F76E5DEC36F0A5D06C5223E0F2CF71F09B
:1089B000F29EAA6A130EA96EA69CA69EA680A85037
:1089C00071BEF28E726EF2CF73F0F29EAA6A140E2E
:1089D000A96EA69CA69EA680A85073BEF28E746E49
:1089E00072C076F074C075F076C078F075C077F01C
:1089F00003DD3BD56B52D8B46FD095DD0152FDE05D
:108A0000990EED6FBFDD0400F90E006E002EFED74B
:108A10000000010E6D6E6D5003082BE3036A6D506C
:108A2000040FE96E000E0320EA6EEFCF71F071C003
:108A3000EDF0A8DD036A6D500C0F016E000E0322ED
:108A400003C072F0036A6D50040FE96E000E03203C
:108A5000EA6EEFCF73F072C0EAFF01C0E9FF73C0A6
:108A6000EFFF0400F90E006E002EFED700006D2A05
:108A7000D2D7810E0C6E010E106E300E116E100EDC
:108A8000126E51DD0152FDE0010EEB6F3CDE4890AD
:108A90006D6A6D50060820E3036A6D500C0FE96E95
:108AA000000E0320EA6EEFCF71F0036A6D50040FE1
:108AB000E96E000E0320EA6EEF50715C0BE0D60EFB
:108AC000F66E640EF76E5DEC36F004009EAAFDD7DC
:108AD000AE500FD06D2ADDD76A5206E0010E716EDE
:108AE000726A736E54DE05D0716A726A010E736E1B
:108AF0004EDE000C200EED6FB5EC39F002C068F0D0
:108B000001C067F0673C03D0683C01D004D06752D5
:108B100004E1685202E1669001D06680EFEC39F022
:108B2000015201E19CD157EC3BF0015207E1140ED8
:108B3000F66E650EF76E5DEC36F091D10D0E040009
:108B40009EA8FDD7AD6E0A0E04009EA8FDD7AD6E9F
:108B50006550F70FD8B05BD1090F30EF47F0668250
:108B60006684475005E0010A07E0030A09E00CD0DB
:108B7000696A91EC3BF00BD0696A9BEC3DF007D041
:108B8000696AA2EC3FF003D0696A91EC3BF03FD1F7
:108B900066826684475005E0010A08E0030A0BE09C
:108BA0000FD0010E696E91EC3BF00ED0010E696E94
:108BB0009BEC3DF009D0010E696EA2EC3FF004D0B1
:108BC000010E696E91EC3BF022D1668266844750BB
:108BD00005E0010A08E0030A0BE00FD0020E696EFF
:108BE00091EC3BF00ED0020E696E9BEC3DF009D08B
:108BF000020E696EA2EC3FF004D0020E696E91EC99
:108C00003BF005D166826684475005E0010A08E022
:108C1000030A0BE00FD0030E696E91EC3BF00ED00F
:108C2000030E696E9BEC3DF009D0030E696EA2EC59
:108C30003FF004D0030E696E91EC3BF0E8D0668201
:108C40006684475005E0010A08E0030A0BE00FD0F4
:108C5000040E696E91EC3BF00ED0040E696E9BEC35
:108C60003DF009D0040E696EA2EC3FF004D0040E72
:108C7000696E91EC3BF0CBD066826684475005E08C
:108C8000010A08E0030A0BE00FD0050E696E91ECB3
:108C90003BF00ED0050E696E9BEC3DF009D0050E41
:108CA000696EA2EC3FF004D0050E696E91EC3BF0CA
:108CB000AED066926694475005E0010A08E0030AC8
:108CC0000BE00FD0060E696E91EC3BF00ED0060E55
:108CD000696E9BEC3DF009D0060E696EA2EC3FF088
:108CE00004D0060E696E91EC3BF00D0E1B6E570E14
:108CF0001A6E0D0E1F6E570E1E6E216A070E206E25
:108D0000A10E236E200E226E296A286A2B6A2A6A17
:108D10000D0E2F6E570E2E6E336A326A376A366A20
:108D20003F6A3E6A74D066826694475005E0010A45
:108D300008E0030A0BE00FD0070E696E91EC3BF0E0
:108D40000ED0070E696E9BEC3DF009D0070E696EE0
:108D5000A2EC3FF004D0070E696E91EC3BF0090ED7
:108D60001B6E0B0E1A6E090E1F6E0B0E1E6E216A05
:108D7000070E206EA10E236E200E226E296A286A2D
:108D80002B6A2A6A090E2F6E0B0E2E6E336A326A18
:108D9000376A366A3F6A3E6A3AD0669266944750AE
:108DA00005E0010A08E0030A0BE00FD0080E696E27
:108DB00091EC3BF00ED0080E696E9BEC3DF009D0B3
:108DC000080E696EA2EC3FF004D0080E696E91ECBB
:108DD0003BF00D0E1B6E110E1A6E0D0E1F6E110E56
:108DE0001E6E216A070E206EA10E236E200E226ECB
:108DF000296A286A2B6A2A6A0D0E2F6E110E2E6EB2
:108E0000336A326A376A366A3F6A3E6A00D066A2BF
:108E100014D066A409D0000E66B0010E6A6E010E71
:108E20006B6E6C6E83DD08D0000E66B0010E6A6E4C
:108E3000010E6B6E6C6A7ADD12D066A409D0000E4A
:108E400066B0010E6A6E6B6A010E6C6E6FDD07D044
:108E5000000E66B0010E6A6E6B6A6C6A67DD000C0C
:108E6000E824F76AF7367B0FF66E8E0EF7220A00BB
:108E7000F550FA6E0800F550F96E5E8B908BCA8B38
:108E8000048C3E8C788CB28C268D9A8DF0C0F1F0DB
:108E9000040EF26F010EF36FF351050805E3D8904D
:108EA000F137F237F32BF8D793928A82939C8A8C0E
:108EB000939A8A8A010EF36FF35109080EE3D89052
:108EC000F137F23702E28A9601D08A869396939818
:108ED0008A8893988A98F32BEFD793968A969392E1
:108EE0008A92939C8A9C939A8A9A7EEF47F0030E0B
:108EF000F36FDFEC3AF0C00EF06FC8D7FF0EEB6FE8
:108F0000070EEC6F010EED6FED51050805E3D890EB
:108F1000EB37EC37ED2BF8D793928A82939C8A8CAF
:108F2000939A8A8A010EED6FED5109080EE3D890ED
:108F3000EB37EC3702E28A9601D08A8693969398B3
:108F40008A8893988A98ED2BEFD793968A96939276
:108F50008A92939C8A9C939A8A9A0400070E006EC8
:108F6000002EFED700D0939A8A8AEF6BEE6BEE3D0F
:108F700003D0EF3D01D00FD0938481A408D0939A01
:108F80008A9AF36BDFEC3AF0010E016E0BD0EE2BF8
:108F9000D8B4EF2BECD7939A8A9AF36BDFEC3AF0C4
:108FA000000E016EC0EF49F0676A666AEA91656A71
:108FB00065503F081AE3D8906534036A680F016E64
:108FC000000E032201C0EBF003C0ECF065C0EDF031
:108FD000B5EC39F0ECC0EAFFEBC0E9FF02C0ECFFF2
:108FE000ED5201C0EFFF652AE3D7A83D03D0A93DAC
:108FF00001D001D0EA8148B009D048EC36F0560ED5
:10900000F66E650EF76E5DEC36F005D0200E0400AE
:109010009EA8FDD7AD6E656A65503F08D8A0A8D060
:1090200048B076D06550070B44E1D8906534036AA8
:10903000680FE96E000E0320EA6EECCFECF0ED5203
:10904000EFCFEBF0ECC0EBF0EC6BD8906534036A3B
:10905000680FE96E000E0320EA6EECCFEEF0ED52E1
:10906000EFCFEDF00D0E04009EA8FDD7AD6E0A0EF9
:1090700004009EA8FDD7AD6E65C0EFF0370EF06F0F
:1090800012EC42F0200E04009EA8FDD7AD6EEBC09E
:10909000EFF0370EF06F12EC42F0EDC0EFF0370E4C
:1090A000F06F12EC42F0200E04009EA8FDD7AD6ECA
:1090B0002ED0D8906534036A680FE96E000E032045
:1090C000EA6EECCFECF0ED52EFCFEBF0ECC0EBF052
:1090D000EC6BD8906534036A680FE96E000E0320CC
:1090E000EA6EECCFEEF0ED52EFCFEDF0EBC0EFF02B
:1090F000370EF06F12EC42F0EDC0EFF0370EF06F6C
:1091000012EC42F0200E04009EA8FDD7AD6E2ED0CA
:10911000D8906534036A680FE96E000E0320EA6E8A
:10912000ECCFECF0ED52EFCFEBF0ECC0EBF0EC6BF2
:10913000D8906534036A680FE96E000E0320EA6E6A
:10914000ECCFEEF0ED52EFCFEDF0EBC0EFF0370EDD
:10915000F06F12EC42F0EDC0EFF0370EF06F12EC52
:1091600042F0200E04009EA8FDD7AD6E652A54D7AC
:10917000840EF66E650EF76E5DEC36F0920EF66EAE
:10918000650EF76E5DEC36F09E0EF66E650EF76EB0
:109190005DEC36F068C000F06950036E02E10052E9
:1091A0002CE0100E035C02E100522EE0200E035C66
:1091B00002E1005230E0300E035C02E1005232E086
:1091C000400E035C02E1005234E0500E035C02E109
:1091D000005236E0F00E035C03E1040E005C37E061
:1091E000F00E035C03E1050E005C38E0F00E035C5A
:1091F00003E1060E005C39E03FD0AA0EF66E650E64
:10920000F76E5DEC36F03ED0B00EF66E650EF76E82
:109210005DEC36F037D0B60EF66E650EF76E5DEC8F
:1092200036F030D0BE0EF66E650EF76E5DEC36F0A1
:1092300029D0C60EF66E650EF76E5DEC36F022D0C4
:10924000D20EF66E650EF76E5DEC36F01BD0E00EBA
:10925000F66E650EF76E5DEC36F014D0EA0EF66E23
:10926000650EF76E5DEC36F00DD0F60EF66E650EFF
:10927000F76E5DEC36F006D0FC0EF66E650EF76EFE
:109280005DEC36F06A506B10000ED8A4010AE86F4E
:10929000E96B160EF66E660EF76E5DEC36F06AC080
:1092A00000F06BC003F0110E6B5C02E100520DE0A8
:1092B000110E035C03E1010E005C0EE0110E035C75
:1092C00003E1020E005C0FE015D0240EF66E660E70
:1092D000F76E5DEC36F014D0340EF66E660EF76E57
:1092E0005DEC36F00DD0400EF66E660EF76E5DEC5E
:1092F00036F006D04E0EF66E660EF76E5DEC36F06A
:109300006850040803E16950F00806E06850060858
:1093100004E16950F00801E1C0D0EB6B83EC43F04D
:10932000015207E1600EF66E660EF76E5DEC36F0E8
:10933000B4D00450810806E09A0EF66E660EF76E01
:109340005DEC36F00D0E04009EA8FDD7AD6E0A0E42
:1093500004009EA8FDD7AD6E6FC0ECF06EC0EBF0C0
:10936000ED6B20EC37F0CA0EF66E660EF76E5DEC14
:1093700036F0F40EF66E660EF76E5DEC36F0B7D58D
:10938000015207E0200EF66E670EF76E5DEC36F0C8
:1093900007D0300EF66E670EF76E5DEC36F07DD0BE
:1093A000656A6550170811E3D8906534036A680F41
:1093B000E96E000E0320EA6EECCF03F0ED52EF50A1
:1093C000662603506722652AECD74C0EF66E670EB0
:1093D000F76E5DEC36F0E651665C03E1E751675CE1
:1093E00056E03F0EEB6F67C0EDF066C0ECF0B4ECFA
:1093F00041F0EA9301B0EA83EAB31DD067C0EBF015
:10940000EC6B600EF66E670EF76E1A0EF26F0FECD5
:1094100037F0EBC0EFF0370EF06F12EC42F066C0A1
:10942000EFF0370EF06F12EC42F02E0E04009EA803
:10943000FDD7AD6E32D0EAA108D03E0EEB6F67C00B
:10944000EDF066C0ECF0B4EC41F067C0EBF0EC6B13
:10945000820EF66E670EF76E0F0EF26F0FEC37F09E
:10946000EBC0EFF0370EF06F12EC42F066C0EFF099
:10947000370EF06F12EC42F00D0E04009EA8FDD7DF
:10948000AD6E0A0E04009EA8FDD7AD6E06D09A0EF2
:10949000F66E670EF76E5DEC36F071EF5FF093904D
:1094A0008A90040000D000D093800400180E006E53
:1094B000002EFED700009380699081B0698004007F
:1094C000B30E006E002EFED70000000E69B0010E34
:1094D000016E000C93908A90040000D000D06A5274
:1094E00008E093800400660E006E002EFED700D0C8
:1094F00007D00400660E006E002EFED700D09380C9
:1095000004006F0E006E002EFED7000C656A666ABE
:10951000676A93EC42F0015203E1000E016E14D130
:10952000F00EED6FC2EC42F066503F08D8A003D1B8
:10953000B6DF689001B068800400A60E006E002EB1
:10954000FED7ADDF689201B0688268A006D068A23D
:1095500004D0678467C001F0F7D068B08AD068B2E1
:1095600088D04650665C1FE16630006E00320032E3
:109570001F0E00160050036A040F016E000E032236
:1095800001C0E9FF03C0EAFF6650070B696E010ED8
:10959000006E6950016E04E0D8900036012EFCD7B1
:1095A0000050EF1244D06650465C22E26630006EF6
:1095B000003200321F0E00160050036A040F016EC5
:1095C000000E032201C0E9FF03C0EAFF6650070B4B
:1095D000696E010E006E6950016E04E0D89000368D
:1095E000012EFCD70050FF0AEF1666C065F01FD0B1
:1095F0006630006E003200321F0E00160050036A03
:10960000040FE96E000E0320EA6EEFCF69F066509A
:10961000070B6A6E69C000F06A50016E04E0D890D2
:109620000032012EFCD700B002D066C065F0663073
:10963000006E003200321F0E00160050036A040F45
:10964000E96E000E0320EA6EEFCF69F06650070B5B
:109650006A6E69C000F06A50016E04E0D890003272
:10966000012EFCD7000E00B0010E6A6E33DF662AB1
:1096700061D068A01FD06630006E003200321F0E2D
:1096800000160050036A040F016E000E032201C091
:10969000E9FF03C0EAFF6650070B696E010E006E1A
:1096A0006950016E04E0D8900036012EFCD70050BE
:1096B000EF121FD06630006E003200321F0E00160F
:1096C0000050036A040F016E000E032201C0E9FF7F
:1096D00003C0EAFF6650070B696E010E006E695009
:1096E000016E04E0D8900036012EFCD70050FF0A2E
:1096F000EF166630006E003200321F0E001600506A
:10970000036A040FE96E000E0320EA6EEFCF69F0E2
:109710006650070B6A6E69C000F06A50016E04E083
:10972000D8900032012EFCD7000E00B0010E6A6EF8
:10973000D1DE662AF9D665C046F0465202E167805E
:1097400001D0678267C001F0A8EF4BF0466ADED611
:109750000150FB0F17E2050FCEEF4BF02E0EF66E09
:10976000640EF76E5DEC36F00DD020EC43F00AD0BD
:1097700020EC43F0ECD74E0EF66E640EF76E5DEC07
:1097800036F000D00A0E04009EA8FDD7AD6E0D0E77
:1097900004009EA8FDD7AD6E71EF5FF0E824F76A74
:1097A000F736B70FF66E970EF7220A00F550FA6EED
:1097B0000800F550F96E5C976A97709784977697D2
:1097C000489048EC36F09A0EF66E690EF76E5DEC36
:1097D00036F004009EAAFDD7AECF65F06550600854
:1097E00006E265507A0803E36550DF0B01D065504F
:1097F000656E6550530A05E01C0A05E00E0A06E096
:1098000008D0476A07D0020E476E04D0010E476E9B
:1098100001D0D9D7AA6A370EA96E47C0A8FFA69C67
:10982000A69EA684F250006EF29E0F01550EA76E02
:10983000AA0EA76EA682A6B2FED7A6940050F21278
:10984000000171EF5FF004009EA8FDD7AD6E000C23
:109850008807896B04009EAAFDD7AECF8AF08A5193
:1098600008080AE1895307E089078A51ECDF200ED6
:10987000EADF8A51E8DF15D08A511F0812E28A51C7
:109880007E080FE38951885D0CE38951892B036AB7
:109890008625E96E87510320EA6E8AC0EFFF8A5160
:1098A000D2DF8A510D08D6E1036A89518625E96E17
:1098B00087510320EA6EEF6A000C8F519119800BDB
:1098C000936F8FAF05D08E1F8F1F8E2BD8B48F2B29
:1098D00091AF05D0901F911F902BD8B4912B8E5132
:1098E0009003F3CF01F0F4CF00F09103F350002682
:1098F0008F519003F3500020026E93AF05D0011EEC
:10990000021E012AD8B4022AF7EF4CF08C6B8A6B46
:109910000A0E8B6F896B886B8651871104E1000EEC
:10992000016E026EE6D08C518C2B036A8625E96E9F
:1099300087510320EA6EEFCF8DF08D512D080DE198
:10994000010E8A6F8C518C2B036A8625E96E875134
:109950000320EA6EEFCF8DF00DD08D512B080AE178
:109960008C518C2B036A8625E96E87510320EA6EA1
:10997000EFCF8DF08D512F08D8B0ADD08D51390873
:10998000D8A0A9D08D51300821E1036A8C518625D9
:10999000E96E87510320EA6EEF5078080AE0036A07
:1099A0008C518625E96E87510320EA6EEF505808E6
:1099B0000DE1100E8B6F8C2B8C518C2B036A86253E
:1099C000E96E87510320EA6EEFCF8DF08B510A08C4
:1099D00021E18D512F081DE28D5139081AE38F6B5B
:1099E0000A0E8E6F89C091F088C090F066D7300E55
:1099F0008D5D0124886F000E0220896F8C518C2BA5
:109A0000036A8625E96E87510320EA6EEFCF8DF059
:109A1000E0D761D08B5110085EE18D51600806E2FD
:109A20008D517A0803E38D51DF0B01D08D518D6F7D
:109A30008D512F0803E28D51390806E28D514008FF
:109A40004AE28D51460847E38D512F0819E28D51A6
:109A5000390816E388358E6F89358F6F8E378F37CB
:109A60008E378F378E378F37F00E8E17300E8D5D15
:109A70008E25016E000E8F2101C088F0896F16D0EF
:109A800088358E6F89358F6F8E378F378E378F374A
:109A90008E378F37F00E8E17410E8D5D0A0F8E2593
:109AA000016E000E8F2101C088F0896F8C518C2BC4
:109AB000036A8625E96E87510320EA6EEF508D6FA9
:109AC000600806E28D517A0803E38D51DF0B01D067
:109AD0008D518D6FADD78B510A0807E18A2D05D0C6
:109AE000881F891F882BD8B4892B88C001F089C0B2
:109AF00002F085EF4DF0876B7D0E866F070E886F45
:109B0000A7DE876B7D0E866F01D702C085F001C08E
:109B100084F084C001F085C002F0000C006A016A84
:109B20007950D8907AB00026003201327AB20026FD
:109B3000003201327AB40026003201327AB60026B1
:109B4000003201327AB80026003201327ABA002699
:109B5000003201327ABC0026003201327ABE002681
:109B60000032013220EF4EF0776A756A0A0E766E87
:109B7000746A7250731003E1000E016EC1D0775009
:109B8000772A036A7224E96E73500320EA6EEFCFDE
:109B900078F078502D080DE1010E756E7750772A18
:109BA000036A7224E96E73500320EA6EEFCF78F0F7
:109BB0000DD078502B080AE17750772A036A722477
:109BC000E96E73500320EA6EEFCF78F078502F08DB
:109BD000D8B08ED078503908D8A08AD078503008C4
:109BE00021E1036A77507224E96E73500320EA6E14
:109BF000EF5078080AE0036A77507224E96E7350D8
:109C00000320EA6EEF5058080DE1100E766E772AA9
:109C10007750772A036A7224E96E73500320EA6E44
:109C2000EFCF78F076500A081BE178502F0817E242
:109C30007850390814E30A0E796E74C07AF06ED742
:109C4000300E785C0124746E7750772A036A722490
:109C5000E96E73500320EA6EEFCF78F0E6D748D074
:109C60007650100845E17850600806E278507A088E
:109C700003E37850DF0B01D07850786E78502F08CE
:109C800003E27850390806E27850400831E2785013
:109C900046082EE378502F080CE27850390809E383
:109CA0007438796EF00E7916300E785C7924746E03
:109CB00009D07438796EF00E7916410E785C0A0F6F
:109CC0007924746E7750772A036A7224E96E735090
:109CD0000320EA6EEFCF78F07850600806E2785003
:109CE0007A0803E37850DF0B01D07850786EC6D73E
:109CF000752C04D076500A0801E1746C74C001F030
:109D00008CEF4EF0876B6C0E866F050E886FA0DDB2
:109D1000736A6C0E726E28D701C071F071C001F0C9
:109D2000E9EF4EF0666A656A489048EC36F0CC0E72
:109D3000F66E680EF76E5DEC36F0DDDE02C06AF09E
:109D400001C069F06A50070804E30BE16950D608C6
:109D500008E26A50060806E2FF0A03E16950E108DA
:109D600001E2E5D7D00E695C656E070E6A58666E33
:109D7000D89065C066F0656A6636F20EF66E680EBB
:109D8000F76E5DEC36F0B7DE02C068F001C067F038
:109D9000675202E1685205E0685203E167500C081F
:109DA00001E2EBD76736683667366836673668365D
:109DB0006736683667366836E00E67166750651294
:109DC00068506612160EF66E690EF76E5DEC36F090
:109DD00099D701C06BF06B5203E06B501F0801E292
:109DE000F1D76B506526000E662266C06CF06D6A76
:109DF000AA6A130EA96E6CC0A8FFA69CA69EA68494
:109E0000F250006EF29E0F01550EA76EAA0EA76EBD
:109E1000A682A6B2FED7A6940050F212AA6A140E29
:109E2000A96E65C0A8FFA69CA69EA684F2CF00F0EE
:109E3000F29E550EA76EAA0EA76EA682A6B2FED7F8
:109E4000A6940050F212380EF66E690EF76E0001FD
:109E50005DEC36F066C06CF06D6A560EF66E690EFB
:109E6000F76E3B0EF26F0FEC37F06CC0EFF0370E71
:109E7000F06F12EC42F065C0EFF0370EF06F12ECAD
:109E800042F00D0E04009EA8FDD7AD6E0A0E040030
:109E90009EA8FDD7AD6E71EF5FF06B6A6A6A48905D
:109EA000C00EF66E690EF76E5DEC36F004009EAAE9
:109EB000FDD7AE50F20EF66E690EF76E5DEC36F021
:109EC00004009EAAFDD7AECF66F06650600806E299
:109ED00066507A0803E36650DF0B01D06650666E69
:109EE0006650590805E066504E08D8A457EF55F063
:109EF0002E0EF66E6A0EF76E5DEC36F093EC42F0C5
:109F00000152FCE00400DD0EEF6F85EC42F0330EF1
:109F1000ED6FC2EC42F0656A6550070819E3040072
:109F2000A60E006E002EFED7036A6550040F016E68
:109F3000000E032201C06EF003C06FF0FDEC42F092
:109F40006FC0EAFF6EC0E9FF01C0EFFF652AE4D7EA
:109F5000656A655007082FE3800E65246E6E010E5A
:109F60006F6ED8B06F2A036A6550040FE96E000E59
:109F70000320EA6EEFCF70F06FC0AAFF6EC0A9FF9A
:109F800070C0A8FFA69CA69EA684F250006EF29E0A
:109F90000F01550EA76EAA0EA76EA682A6B2FED717
:109FA000A6940050F2122E0E04009EA8FDD7AD6EAE
:109FB000652A0001CED7656A65503F084DE365C04C
:109FC000EDF0B5EC39F002C069F001C068F0D8904E
:109FD00065346E6E010E6F6E69C070F0716A6FC08D
:109FE000AAFF6EC0A9FF70C0A8FFA69CA69EA6846B
:109FF000F250006EF29E0F01550EA76EAA0EA76ECC
:10A00000A682A6B2FED7A6940050F212D89065346C
:10A01000010F6E6E010E6F6ED8B06F2A6FC0AAFF6F
:10A020006EC0A9FF68C0A8FFA69CA69EA684F2CF1A
:10A0300000F0F29E550EA76EAA0EA76EA682A6B2DB
:10A04000FED7A6940050F2122E0E04009EA8FDD753
:10A05000AD6E652A0001B0D766505908D8A490EFBC
:10A0600054F0520EF66E6A0EF76E5DEC36F0860E08
:10A07000F66E6A0EF76E5DEC36F004009EAAFDD710
:10A08000AECF67F06750300803E26750360801E250
:10A09000E3D7310E675CF70FD8B091D1090F5BEFB2
:10A0A00055F0010EAA6EA96AA86AA69CA69EA6846F
:10A0B000F250006EF29E0F01550EA76EAA0EA76E0B
:10A0C000A682A6B2FED7A6940050F212010EAA6E86
:10A0D000A96EA86AA69CA69EA684F250006EF29E67
:10A0E000550EA76EAA0EA76EA682A6B2FED7A6949C
:10A0F0000050F212000163D1010EAA6EA96A100E7F
:10A10000A86EA69CA69EA684F250006EF29E0F0139
:10A11000550EA76EAA0EA76EA682A6B2FED7A6946B
:10A120000050F212010EAA6EA96EA86AA69CA69E05
:10A13000A684F250006EF29E550EA76EAA0EA76E70
:10A14000A682A6B2FED7A6940050F212000137D123
:10A15000010EAA6EA96A200EA86EA69CA69EA684D1
:10A16000F250006EF29E0F01550EA76EAA0EA76E5A
:10A17000A682A6B2FED7A6940050F212010EAA6ED5
:10A18000A96EA86AA69CA69EA684F250006EF29EB6
:10A19000550EA76EAA0EA76EA682A6B2FED7A694EB
:10A1A0000050F21200010BD1010EAA6EA96A300E06
:10A1B000A86EA69CA69EA684F250006EF29E0F0189
:10A1C000550EA76EAA0EA76EA682A6B2FED7A694BB
:10A1D0000050F212010EAA6EA96EA86AA69CA69E55
:10A1E000A684F250006EF29E550EA76EAA0EA76EC0
:10A1F000A682A6B2FED7A6940050F2120001DFD0CC
:10A20000010EAA6EA96A400EA86EA69CA69EA68400
:10A21000F250006EF29E0F01550EA76EAA0EA76EA9
:10A22000A682A6B2FED7A6940050F212010EAA6E24
:10A23000A96EA86AA69CA69EA684F250006EF29E05
:10A24000550EA76EAA0EA76EA682A6B2FED7A6943A
:10A250000050F2120001B3D0010EAA6EA96A500E8E
:10A26000A86EA69CA69EA684F250006EF29E0F01D8
:10A27000550EA76EAA0EA76EA682A6B2FED7A6940A
:10A280000050F212010EAA6EA96EA86AA69CA69EA4
:10A29000A684F250006EF29E550EA76EAA0EA76E0F
:10A2A000A682A6B2FED7A6940050F212000187D073
:10A2B000010EAA6EA96AF00EA86EA69CA69EA684A0
:10A2C000F250006EF29E0F01550EA76EAA0EA76EF9
:10A2D000A682A6B2FED7A6940050F212010EAA6E74
:10A2E000A96E040EA86EA69CA69EA684F250006ECF
:10A2F000F29E550EA76EAA0EA76EA682A6B2FED734
:10A30000A6940050F21200015AD0010EAA6EA96A5A
:10A31000F00EA86EA69CA69EA684F250006EF29E39
:10A320000F01550EA76EAA0EA76EA682A6B2FED783
:10A33000A6940050F212010EAA6EA96E050EA86E28
:10A34000A69CA69EA684F250006EF29E550EA76EA5
:10A35000AA0EA76EA682A6B2FED7A6940050F2124D
:10A3600000012DD0010EAA6EA96AF00EA86EA69C5F
:10A37000A69EA684F250006EF29E0F01550EA76EA7
:10A38000AA0EA76EA682A6B2FED7A6940050F2121D
:10A39000010EAA6EA96E060EA86EA69CA69EA684A5
:10A3A000F250006EF29E550EA76EAA0EA76EA68200
:10A3B000A6B2FED7A6940050F212000100D0010E02
:10A3C000AA6E0C0EA96EA86AA69CA69EA684F25040
:10A3D000006EF29E0F01550EA76EAA0EA76EA68202
:10A3E000A6B2FED7A6940050F212010EAA6E0D0E70
:10A3F000A96E0F0EA86EA69CA69EA684F2CF00F0B2
:10A40000F29E550EA76EAA0EA76EA682A6B2FED722
:10A41000A6940050F212010EAA6E0E0EA96E420E04
:10A42000A86EA69CA69EA684F2CF00F0F29E550EC2
:10A43000A76EAA0EA76EA682A6B2FED7A69400505B
:10A44000F212010EAA6E0F0EA96E400EA86EA69C07
:10A45000A69EA684F2CF00F0F29E550EA76EAA0E1D
:10A46000A76EA682A6B2FED7A6940050F212010EE5
:10A47000AA6E140EA96EA86AA69CA69EA684F2CF08
:10A4800000F0F29E550EA76EAA0EA76EA682A6B287
:10A49000FED7A6940050F212010EAA6E150EA96EF8
:10A4A000A86AA69CA69EA684F2CF00F0F29E550E46
:10A4B000A76EAA0EA76EA682A6B2FED7A6940050DB
:10A4C000F212010EAA6E160EA96EA86AA69CA69E8E
:10A4D000A684F2CF00F0F29E550EA76EAA0EA76ECC
:10A4E000A682A6B2FED7A6940050F212010EAA6E62
:10A4F000170EA96EA86AA69CA69EA684F2CF00F0AD
:10A50000F29E550EA76EAA0EA76EA682A6B2FED721
:10A51000A6940050F212010EAA6E1E0EA96EA86A31
:10A52000A69CA69EA684F2CF00F0F29E550EA76EC2
:10A53000AA0EA76EA682A6B2FED7A6940050F2126B
:10A54000010EAA6E1F0EA96EA86AA69CA69EA684DE
:10A55000F2CF00F0F29E550EA76EAA0EA76EA6824D
:10A56000A6B2FED7A6940050F212010EAA6E220ED9
:10A57000A96EA86AA69CA69EA684F2CF00F0F29EC1
:10A58000550EA76EAA0EA76EA682A6B2FED7A694F7
:10A590000050F212010EAA6E230EA96EA86AA69CA4
:10A5A000A69EA684F2CF00F0F29E550EA76EAA0ECC
:10A5B000A76EA682A6B2FED7A6940050F212010E94
:10A5C000AA6E260EA96EFF0EA86EA69CA69EA68455
:10A5D000F2CF00F0F29E550EA76EAA0EA76EA682CD
:10A5E000A6B2FED7A6940050F212010EAA6E270E54
:10A5F000A96EFF0EA86EA69CA69EA684F2CF00F0C0
:10A60000F29E550EA76EAA0EA76EA682A6B2FED720
:10A61000A6940050F212010EAA6E2A0EA96EA86A24
:10A62000A69CA69EA684F2CF00F0F29E550EA76EC1
:10A63000AA0EA76EA682A6B2FED7A6940050F2126A
:10A64000010EAA6E2B0EA96EA86AA69CA69EA684D1
:10A65000F2CF00F0F29E550EA76EAA0EA76EA6824C
:10A66000A6B2FED7A6940050F212010EAA6E2C0ECE
:10A67000A96EFF0EA86EA69CA69EA684F2CF00F03F
:10A68000F29E550EA76EAA0EA76EA682A6B2FED7A0
:10A69000A6940050F212010EAA6E2D0EA96EFF0EA6
:10A6A000A86EA69CA69EA684F2CF00F0F29E550E40
:10A6B000A76EAA0EA76EA682A6B2FED7A6940050D9
:10A6C000F212F2CF6EF0F29EAA6A130EA96EA69C49
:10A6D000A69EA680A8506EBEF28E656E010EAA6E72
:10A6E000060EA96E65C0A8FFA69CA69EA684F2CF02
:10A6F00000F0F29E550EA76EAA0EA76EA682A6B215
:10A70000FED7A6940050F212010EAA6E0A0EA96E90
:10A7100065C0A8FFA69CA69EA684F2CF00F0F29E7C
:10A72000550EA76EAA0EA76EA682A6B2FED7A69455
:10A730000050F212010EAA6E1A0EA96E65C0A8FF93
:10A74000A69CA69EA684F2CF00F0F29E550EA76EA0
:10A75000AA0EA76EA682A6B2FED7A6940050F21249
:10A76000F2CF6EF0F29EAA6A140EA96EA69CA69E67
:10A77000A680A8506EBEF28E656E010EAA6E070E00
:10A78000A96E65C0A8FFA69CA69EA684F2CF00F085
:10A79000F29E550EA76EAA0EA76EA682A6B2FED78F
:10A7A000A6940050F212010EAA6E0B0EA96E65C09F
:10A7B000A8FFA69CA69EA684F2CF00F0F29E550E9E
:10A7C000A76EAA0EA76EA682A6B2FED7A6940050C8
:10A7D000F212010EAA6E1B0EA96E65C0A8FFA69C00
:10A7E000A69EA684F2CF00F0F29E550EA76EAA0E8A
:10A7F000A76EA682A6B2FED7A6940050F212010E52
:10A800006D6E300E6C6E6D5001081EE303E16C50EE
:10A810007D081AE36DC0AAFF6CC0A9FFFF0EA86EE9
:10A82000A69CA69EA684F2CF00F0F29E550EA76EBF
:10A83000AA0EA76EA682A6B2FED7A6940050F21268
:10A840006C2AD8B46D2ADFD7010E6D6E6C6A6D501C
:10A85000010835E303E16C502F0831E36B6A6A6A43
:10A86000F2CF6EF0F29E6DC0AAFF6CC0A9FFA69C4D
:10A87000A69EA680A8506EBEF28E6F6E010E6C244E
:10A88000706E000E6D20716EF2CF72F0F29E71C08C
:10A89000AAFF70C0A9FFA69CA69EA680A85072BE63
:10A8A000F28E706E6FC069F070C068F068506A26F2
:10A8B00069506B22020E6C26000E6D22C8D76BC049
:10A8C0006EF06F6A010EAA6E7E0EA96E6BC0A8FFB5
:10A8D000A69CA69EA684F2CF00F0F29E550EA76E0F
:10A8E000AA0EA76EA682A6B2FED7A6940050F212B8
:10A8F000010EAA6E7F0EA96E6AC0A8FFA69CA69E36
:10A90000A684F2CF00F0F29E550EA76EAA0EA76E97
:10A91000A682A6B2FED7A6940050F212C0D00001C3
:10A92000F2CF6EF0F29E010EAA6E7C0EA96EA69C6E
:10A93000A69EA680A8506EBEF28E6F6EF2CF70F00B
:10A94000F29E010EAA6E7D0EA96EA69CA69EA68002
:10A95000A85070BEF28E716E6FC073F071C072F04D
:10A96000723C03D0733C01D09BD06B6A6A6A010EC3
:10A970006D6E6C6A6D50010833E303E16C502F0873
:10A980002FE3F2CF6EF0F29E6DC0AAFF6CC0A9FF5C
:10A99000A69CA69EA680A8506EBEF28E6F6E010E7B
:10A9A0006C24706E000E6D20716EF2CF72F0F29E0C
:10A9B00071C0AAFF70C0A9FFA69CA69EA680A85041
:10A9C00072BEF28E706E6FC069F070C068F0685031
:10A9D0006A2669506B22020E6C26000E6D22CAD7C1
:10A9E0006BC06EF06F6A010EAA6E7C0EA96E6EC00F
:10A9F000A8FFA69CA69EA684F250006EF29E0F01B0
:10AA0000550EA76EAA0EA76EA682A6B2FED7A69472
:10AA10000050F212010EAA6E7D0EA96E6AC0A8FF48
:10AA2000A69CA69EA684F2CF00F0F29E550EA76EBD
:10AA3000AA0EA76EA682A6B2FED7A6940050F21266
:10AA40006BC06EF06F6A010EAA6E7E0EA96E6BC0AF
:10AA5000A8FFA69CA69EA684F2CF00F0F29E550EFB
:10AA6000A76EAA0EA76EA682A6B2FED7A694005025
:10AA7000F212010EAA6E7F0EA96E6AC0A8FFA69CF4
:10AA8000A69EA684F2CF00F0F29E550EA76EAA0EE7
:10AA9000A76EA682A6B2FED7A6940050F2120001BD
:10AAA000C60EF66E6A0EF76E5DEC36F002D05AEF07
:10AAB0004FF071EF5FF0E824F76AF736D10FF66ECA
:10AAC000AA0EF7220A00F550FA6E0800F550F96E4A
:10AAD000A2A0F8A050A1A8A100A258A2B0A20AA3C7
:10AAE00064A36A80200EED6FB5EC39F002C06CF003
:10AAF00001C06BF0013C03D06C3C01D00CD0200EA7
:10AB0000ED6FB5EC39F002C06CF001C06BF06B5228
:10AB100004E16C5202E16A9201D06A824890EFEC43
:10AB200039F0015201E1C9D0D40EF66E6A0EF76E0B
:10AB30005DEC36F004009EAAFDD7AE501C0EF66EFA
:10AB40006B0EF76E5DEC36F093EC42F00152FCE0D8
:10AB5000990EED6FC2EC42F00400F90E006E002E6B
:10AB6000FED70000F2CF6BF0F29E010EAA6E810EAE
:10AB7000A96EA69CA69EA680A8506BBEF28E6C6E97
:10AB80006CC0EDF0C2EC42F02E0E04009EA8FDD782
:10AB9000AD6E0400F90E006E002EFED70000F2CF5D
:10ABA0006BF0F29E010EAA6E820EA96EA69CA69E66
:10ABB000A680A8506BBEF28E6C6E6CC0EDF0C2EC3D
:10ABC00042F02E0E04009EA8FDD7AD6E0400F90ED3
:10ABD000006E002EFED70000F2CF6BF0F29E010E49
:10ABE000AA6E830EA96EA69CA69EA680A8506BBED8
:10ABF000F28E6C6E6CC0EDF0C2EC42F02E0E0400D2
:10AC00009EA8FDD7AD6E020E6B6E960EED6F2FEC0B
:10AC100036F06B2EFAD757EC3BF0656A65503F086B
:10AC20004CE3D89065346B6E010E6C6EF2CF6DF014
:10AC3000F29E6CC0AAFF6BC0A9FFA69CA69EA68030
:10AC4000A8506DBEF28E6B6ED89065346E6E010E9C
:10AC50006F6E010E6E26000E6F22F2CF6CF0F29E28
:10AC60006FC0AAFF6EC0A9FFA69CA69EA680A85092
:10AC70006CBEF28E6E6E6BC067F06EC066F065C023
:10AC8000EBF067C0EDF066C0ECF0B4EC41F02E0ED6
:10AC900004009EA8FDD7AD6E65C0EDF0B5EC39F0AF
:10ACA00002C069F001C068F06650685C03E167505B
:10ACB000695C01E06A90652AB1D771EF5FF0010E1F
:10ACC000D06FD051CF5D07E3CB31CE33CD33CC3312
:10ACD000CB33D02BF6D7CBC000F0CCC001F0CDC029
:10ACE00002F0CEC003F0000C010ED06FD051CF5D4A
:10ACF00007E3CE35CB37CC37CD37CE37D02BF6D791
:10AD0000CBC000F0CCC001F0CDC002F0CEC003F04B
:10AD1000000C120E886F340E876F560E866F780EF9
:10AD2000856F010E836F83510A0837E38351040D49
:10AD3000F350036A850F016E000E032201C0C5F0B7
:10AD400003C0C6F0010E835D040DF350036A850F46
:10AD5000E96E000E0320EA6EEFCFC7F0ECCFC8F02B
:10AD6000ECCFC9F0ECCFCAF0CAC0CEF0C9C0CDF06C
:10AD7000C8C0CCF0C7C0CBF0020ECF6FA0DFC6C0FA
:10AD8000EAFFC5C0E9FF00C0EFFF01C0ECFF02C051
:10AD9000ECFF03C0ECFF832BC6D7F2CFC5F0F29EC9
:10ADA000AA6A200EA96EA69CA69EA680A850C5BF22
:10ADB000F28EC66FF2CFC7F0F29EAA6A210EA96E7C
:10ADC000A69CA69EA680A850C7BFF28EC86F7DC065
:10ADD000B3F07EC0B4F0C6C0B2F0C8C0B1F09A0EF5
:10ADE000B86FBC0EB76FDE0EB66FF00EB56FF2CF58
:10ADF000C5F0F29EAA6A220EA96EA69CA69EA68007
:10AE0000A850C5BFF28EC66FC6C0BCF0FF0EBB6FA8
:10AE1000FF0EBA6F800EB96FC06BBF6BBE6BBD6BA0
:10AE2000C46BC36B010EC26FB80EC16F670E526E5A
:10AE3000450E516E230E506E010E4F6EEF0E566E84
:10AE4000CD0E556EAB0E546E890E536E980E5A6E23
:10AE5000BA0E596EDC0E586EFE0E576E100E5E6EF8
:10AE6000320E5D6E540E5C6E760E5B6EC30E626EBD
:10AE7000D20E616EE10E606EF00E5F6E836B8351D9
:10AE80004F08D8A0AFD283510F0B846F83510F08A6
:10AE9000D8B085D08451040DF350036A850F016E3C
:10AEA000000E032201C0C5F003C0C6F00D0E8425BC
:10AEB0000F0B040DF350036A850FE96E000E03209B
:10AEC000EA6EEFCFC7F0ECCFC8F0ECCFC9F0ECCF13
:10AED000CAF0080E84250F0B040DF350036A850F8A
:10AEE000E96E000E0320EA6EEFCF00F0ECCF01F028
:10AEF000ECCF02F0ECCF03F00050C71B0150C81B91
:10AF00000250C91B0350CA1B020E84250F0B040DEF
:10AF1000F350036A850FE96E000E0320EA6EEFCF4F
:10AF200000F0ECCF01F0ECCF02F0ECCF03F00050DA
:10AF3000C71B0150C81B0250C91B0350CA1B8451B8
:10AF4000040DF350036A850FE96E000E0320EA6ECC
:10AF5000EFCF00F0ECCF01F0ECCF02F0ECCF03F03C
:10AF60000050C71B0150C81B0250C91B0350CA1B0D
:10AF7000CAC0CEF0C9C0CDF0C8C0CCF0C7C0CBF0BD
:10AF8000010ECF6FB1DEC6C0EAFFC5C0E9FF00C049
:10AF9000EFFF01C0ECFF02C0ECFF03C0ECFF8351E8
:10AFA000130802E2000E01D0010E010B78E052C03E
:10AFB000CEF051C0CDF050C0CCF04FC0CBF0050E5C
:10AFC000CF6F92DE03C0C8F002C0C7F001C0C6F068
:10AFD00000C0C5F053505714C96F54505814CA6F6D
:10AFE00055505914CB6F56505A14CC6F53C0CDF0F6
:10AFF000CD1F54C0CEF0CE1F55C0CFF0CF1F56C0CE
:10B00000D0F0D01FCD515B14006ECE515C14016E98
:10B01000CF515D14026ED0515E14036E0050C91101
:10B02000006E0150CA11016E0250CB11026E035026
:10B03000CC11036E0050C5270150C6230250C72310
:10B040000350C8235F50C5276050C6236150C723F3
:10B050006250C8238451040DF350036A850FE96ED2
:10B06000000E0320EA6EEFCF00F0ECCF01F0ECCF42
:10B0700002F0ECCF03F00050C5270150C623025068
:10B08000C7230350C823990EC5257F6E790EC621AC
:10B09000806F820EC721816F5A0EC821826F835143
:10B0A000130802E3000E01D0010EC56F835127087B
:10B0B00002E2000E01D0010EC51560E052C0CEF0D4
:10B0C00051C0CDF050C0CCF04FC0CBF0050ECF6FCB
:10B0D0000BDE03C0C8F002C0C7F001C0C6F000C05C
:10B0E000C5F053505718C96F54505818CA6F55506F
:10B0F0005918CB6F56505A18CC6FC9515B18006E57
:10B10000CA515C18016ECB515D18026ECC515E18AD
:10B11000036E0050C5270150C6230250C7230350B9
:10B12000C8235F50C5276050C6236150C7236250B3
:10B13000C8238451040DF350036A850FE96E000E95
:10B140000320EA6EEFCF00F0ECCF01F0ECCF02F07D
:10B15000ECCF03F00050C5270150C6230250C7238F
:10B160000350C823A10EC5257F6EEB0EC621806F4C
:10B17000D90EC721816F6E0EC821826F83512708B7
:10B1800002E3000E01D0010EC56F83513B0802E2BD
:10B19000000E01D0010EC515D8B480D052C0CEF03B
:10B1A00051C0CDF050C0CCF04FC0CBF0050ECF6FEA
:10B1B0009BDD03C0C8F002C0C7F001C0C6F000C0EC
:10B1C000C5F053505714C96F54505814CA6F555096
:10B1D0005914CB6F56505A14CC6F53505B14006EF9
:10B1E00054505C14016E55505D14026E56505E143E
:10B1F000036E0050C9130150CA130250CB13035001
:10B20000CC1357505B14006E58505C14016E5950AB
:10B210005D14026E5A505E14036E0050C911006E28
:10B220000150CA11016E0250CB11026E0350CC11B5
:10B23000036E0050C5270150C6230250C723035098
:10B24000C8235F50C5276050C6236150C723625092
:10B25000C8238451040DF350036A850FE96E000E74
:10B260000320EA6EEFCF00F0ECCF01F0ECCF02F05C
:10B27000ECCF03F00050C5270150C6230250C7236E
:10B280000350C823DC0EC5257F6EBC0EC621806F1F
:10B290001B0EC721816F8F0EC821826F83513B081F
:10B2A00002E3000E01D0010EC56F83514F0802E288
:10B2B000000E01D0010EC51560E052C0CEF051C0A5
:10B2C000CDF050C0CCF04FC0CBF0050ECF6F0CDDF1
:10B2D00003C0C8F002C0C7F001C0C6F000C0C5F08E
:10B2E00053505718C96F54505818CA6F55505918B1
:10B2F000CB6F56505A18CC6FC9515B18006ECA51AB
:10B300005C18016ECB515D18026ECC515E18036E55
:10B310000050C5270150C6230250C7230350C8233D
:10B320005F50C5276050C6236150C7236250C823B1
:10B330008451040DF350036A850FE96E000E03205B
:10B34000EA6EEFCF00F0ECCF01F0ECCF02F0ECCFE3
:10B3500003F00050C5270150C6230250C7230350F5
:10B36000C823D60EC5257F6EC10EC621806F620E22
:10B37000C721816FCA0EC821826F5EC062F05DC0B6
:10B3800061F05CC060F05BC05FF05AC05EF059C015
:10B390005DF058C05CF057C05BF056C0CEF055C0B1
:10B3A000CDF054C0CCF053C0CBF0020ECF6F87DC91
:10B3B00003C05AF002C059F001C058F000C057F065
:10B3C00052C056F051C055F050C054F04FC053F029
:10B3D00082C052F081C051F080C050F07FC04FF069
:10B3E000832B4DD5E1EF5AF004009EAAFDD7AECFD6
:10B3F00082F0825123EC4CF08251390805E3300E83
:10B40000825D016E0FD00ED08251600806E282513B
:10B410007A0803E38251DF0B01D08251BF0F0A0F7C
:10B42000016E00D0000CE0DF01C081F0DDDF01C063
:10B4300080F08051DD0804E181C001F007D006D022
:10B440008151100DF3508025016E00D0000C48ECA6
:10B4500036F0F2CF7DF0F29EAA6A200EA96EA69C6D
:10B46000A69EA680A8507DBEF28E7E6EF2CF7FF0A3
:10B47000F29EAA6A210EA96EA69CA69EA680A8503E
:10B480007FBEF28E806F7EC082F080C081F0F2CFEE
:10B4900083F0F29EAA6A220EA96EA69CA69EA680A2
:10B4A000A85083BFF28E846F4A0EF66E600EF76E60
:10B4B000150EF26F0FEC37F0100EE96E82C0F3F04C
:10B4C00081C0F2F0BCEC36F0620EF66E600EF76EE4
:10B4D0000D0EF26F0FEC37F084C0F2F01B0EF36F1D
:10B4E00083EC36F00D0E04009EA8FDD7AD6E0A0E5B
:10B4F00004009EA8FDD7AD6E0A0E04009EA8FDD7DD
:10B50000AD6E760EF66E600EF76E5DEC36F0C40E24
:10B51000F66E600EF76E5DEC36F0F2CF7DF0F29EC7
:10B52000AA6A100EA96EA69CA69EA680A8507DBEF3
:10B53000F28E7E6EF2CF7FF0F29EAA6A110EA96E95
:10B54000A69CA69EA680A8507FBEF28E806F7EC06D
:10B5500068F080C067F0120EF66E610EF76E130E83
:10B56000F26F0FEC37F0100EE96E68C0F3F067C0B1
:10B57000F2F0BCEC36F00D0E04009EA8FDD7AD6EC7
:10B580000A0E04009EA8FDD7AD6E0A0E04009EA808
:10B59000FDD7AD6E2C0EF66E610EF76E5DEC36F0DB
:10B5A0007BEC4DF002C066F001C065F0655203E12E
:10B5B000665201E14CD166C07EF065C07DF089EF36
:10B5C00056F0640EF66E610EF76E5DEC36F0EC0E22
:10B5D000F66E5E0EF76E5DEC36F0920EF66E610E54
:10B5E000F76E5DEC36F01FDF01C07DF01CDF01C09F
:10B5F0007EF019DF01C07FF016DF7DC06CF07EC0E9
:10B600006BF07FC06AF001C069F00DDF01C07DF012
:10B610000ADF01C07EF007DF01C07FF004DF7DC0DC
:10B6200070F07EC06FF07FC06EF001C06DF0FBDE89
:10B6300001C07DF0F8DE01C07EF0F5DE01C07FF0D4
:10B64000F2DE7DC074F07EC073F07FC072F001C086
:10B6500071F0E9DE01C07DF0E6DE01C07EF0E3DEE0
:10B6600001C07FF0E0DE7DC078F07EC077F07FC063
:10B6700076F001C075F0D7DE01C07DF0D4DE01C0E8
:10B680007EF0D1DE01C07FF0CEDE7DC07CF07EC0DA
:10B690007BF07FC07AF001C079F04F50695CD8A48C
:10B6A000C8D050506A5CD8A4C4D051506B5CD8A4A8
:10B6B000C0D052506C5CD8A4BCD053506D5CD8A4A0
:10B6C000B8D054506E5CD8A4B4D055506F5CD8A498
:10B6D000B0D05650705CD8A4ACD05750715CD8A490
:10B6E000A8D05850725CD8A4A4D05950735CD8A488
:10B6F000A0D05A50745CD8A49CD05B50755CD8A480
:10B7000098D05C50765CD8A494D05D50775CD8A477
:10B7100090D05E50785CD8A48CD05F50795CD8A46F
:10B7200088D060507A5CD8A484D061507B5CD8A467
:10B7300080D062507C5CD8A47CD06750652668506D
:10B74000662266C07DF07E6AAA6A100EA96E7DC070
:10B75000A8FFA69CA69EA684F250006EF29E0F0142
:10B76000550EA76EAA0EA76EA682A6B2FED7A69405
:10B770000050F212AA6A110EA96E65C0A8FFA69C1D
:10B78000A69EA684F2CF00F0F29E550EA76EAA0EDA
:10B79000A76EA682A6B2FED7A6940050F212F2CFF0
:10B7A0007DF0F29EAA6A220EA96EA69CA69EA68095
:10B7B000A8507DBEF28E010F7E6EAA6A220EA96E7F
:10B7C0007EC0A8FFA69CA69EA684F250006EF29EA4
:10B7D000550EA76EAA0EA76EA682A6B2FED7A69495
:10B7E0000050F212980EF66E610EF76E2B0E0001ED
:10B7F000F26F0FEC37F0100EE96E68C0F3F067C01F
:10B80000F2F0BCEC36F0C60EF66E610EF76E040E6A
:10B81000F26F0FEC37F0100EE96E66C0F3F065C002
:10B82000F2F0BCEC36F02E0E04009EA8FDD7AD6EF3
:10B8300006D0D00EF66E610EF76E5DEC36F0080E97
:10B840007D6EFA0EED6F2FEC36F07D2EFAD771EF8C
:10B850005FF0489048EC36F0CA0EF66E670EF76E51
:10B860005DEC36F0E0DD01C065F0E80EF66E670EC7
:10B87000F76E5DEC36F0D7DD01C066F0D4DD01C0B7
:10B8800067F066C069F067C068F0060EF66E680E75
:10B89000F76E5DEC36F06550030806E0655005086C
:10B8A00003E065500D081BE169C078F068C077F0CF
:10B8B000FCEC41F0240EF66E680EF76E110EF26F7E
:10B8C0000FEC37F066C0EFF0370EF06F12EC42F07D
:10B8D00067C0EFF0370EF06F12EC42F0CED065503B
:10B8E0000B0803E06550200825E10B0EEB6F69C0E3
:10B8F000EDF068C0ECF0B4EC41F0200EEB6F69C0E5
:10B90000EDF068C0ECF0B4EC41F03C0EF66E680E61
:10B91000F76E0E0EF26F0FEC37F066C0EFF0370ED9
:10B92000F06F12EC42F067C0EFF0370EF06F12ECE0
:10B9300042F0A3D065500F0803E06550230825E1CD
:10B940000F0EEB6F69C0EDF068C0ECF0B4EC41F0A5
:10B95000230EEB6F69C0EDF068C0ECF0B4EC41F081
:10B96000520EF66E680EF76E0E0EF26F0FEC37F099
:10B9700066C0EFF0370EF06F12EC42F067C0EFF0E8
:10B98000370EF06F12EC42F078D06550110803E0EA
:10B990006550240825E1110EEB6F69C0EDF068C019
:10B9A000ECF0B4EC41F0240EEB6F69C0EDF068C030
:10B9B000ECF0B4EC41F0680EF66E680EF76E0E0E09
:10B9C000F26F0FEC37F066C0EFF0370EF06F12EC4D
:10B9D00042F067C0EFF0370EF06F12EC42F04DD03E
:10B9E00065500A0803E065501F0825E10A0EEB6F59
:10B9F00069C0EDF068C0ECF0B4EC41F01F0EEB6FE5
:10BA000069C0EDF068C0ECF0B4EC41F07E0EF66E6B
:10BA1000680EF76E0E0EF26F0FEC37F066C0EFF0A7
:10BA2000370EF06F12EC42F067C0EFF0370EF06F98
:10BA300012EC42F022D065C0EBF069C0EDF068C0B6
:10BA4000ECF0B4EC41F065C0EFF0370EF06F12ECA3
:10BA500042F0970EF66E680EF76E070EF26F0FEC5F
:10BA600037F066C0EFF0370EF06F12EC42F067C0AF
:10BA7000EFF0370EF06F12EC42F071EF5FF0F86A02
:10BA8000D09EEA6AE96AB8862A0EAF6E000EB06EE2
:10BA9000A60EAC6E900EAB6E456A446A4890C150DB
:10BAA000C00B0F09C16E070EB46E810E046E056ADD
:10BAB000066A076A010E086E300E096E100E0A6ED5
:10BAC0000B6A146A156A166A176A186A196A1A6A7A
:10BAD0001B6A1C6A1D6A1E6A1F6A206A216A226A22
:10BAE000236A246A256A266A276A286A296A2A6AD2
:10BAF0002B6A2C6A2D6A2E6A2F6A306A316A326A82
:10BB0000336A346A356A366A376A386A396A3A6A31
:10BB10003B6A3C6A3D6A3E6A3F6A406A416A426AE1
:10BB2000436A466A476A496A4A6A646AC150C00BF6
:10BB30000F09C16EC290C69A949A94889496010E89
:10BB4000C66E000EC76ED190800ED56ECD6A000E07
:10BB5000CA6E000ECB6E070EB46E9250926E040049
:10BB6000100E006E002EFED7B450A19CB56A9296BE
:10BB70008996929A899A929E899E94908B901FEFB3
:10BB800036F02CEC36F0640EED6F2FEC36F046EC10
:10BB900036F0F2CF65F0F29EAA6A370EA96EA69C27
:10BBA000A69EA680A85065BEF28E476E4750030839
:10BBB00017E2476AAA6A370EA96EA86AA69CA69ED3
:10BBC000A684F250006EF29E0F01550EA76EAA0ECB
:10BBD000A76EA682A6B2FED7A6940050F21200016C
:10BBE000D19048B070D048EC36F03E0EF66E6B0E39
:10BBF000F76E5DEC36F0920EF66E6B0EF76E5DEC46
:10BC000036F0EC0EF66E5E0EF76E5DEC36F02E0E34
:10BC100004009EA8FDD7AD6E200E04009EA8FDD79F
:10BC2000AD6E520E04009EA8FDD7AD6E530E0400FB
:10BC30009EA8FDD7AD6E410E04009EA8FDD7AD6E47
:10BC40009E0EF66E6B0EF76E5DEC36F0000EF66E25
:10BC50005F0EF76E5DEC36F02E0E04009EA8FDD749
:10BC6000AD6E0D0E04009EA8FDD7AD6E0A0E040049
:10BC70009EA8FDD7AD6EA60EF66E6B0EF76E5DEC50
:10BC800036F0100EF66E5F0EF76E5DEC36F00D0EB0
:10BC900004009EA8FDD7AD6E0A0E04009EA8FDD735
:10BCA000AD6E0D0E04009EA8FDD7AD6E0A0E040009
:10BCB0009EA8FDD7AD6E9FEF37F0B60EF66E6B0EF9
:10BCC000F76E5DEC36F004009EAAFDD7AECF63F0B0
:10BCD0006350600806E263507A0803E36350DF0BA9
:10BCE00001D06350636E6450635C04E0456A010EEA
:10BCF000446E03D0442AD8B4452A2CEC36F0635065
:10BD0000310A31E0030A38E0010A40E0070A48E05E
:10BD1000010A50E0030A58E0010A60E00F0AD8B4B3
:10BD200067D0010AD8B46ED0780AD8B475D0030AA7
:10BD3000D8B47AD0010AD8B47FD0070AD8B484D056
:10BD4000010AD8B489D0030AD8B48ED0010AD8B475
:10BD500093D00F0AD8B498D0010AD8B49CD0030A63
:10BD6000D8B4A3D0B8D0310E04009EA8FDD7AD6ED4
:10BD7000656A7AEC45F0B5D0320E04009EA8FDD776
:10BD8000AD6E010E656E7AEC45F0ABD0330E04005B
:10BD90009EA8FDD7AD6E020E656E7AEC45F0A1D07F
:10BDA000340E04009EA8FDD7AD6E030E656E7AECCE
:10BDB00045F097D0350E04009EA8FDD7AD6E040E59
:10BDC000656E7AEC45F08DD0360E04009EA8FDD746
:10BDD000AD6E050E656E7AEC45F083D0370E04002B
:10BDE0009EA8FDD7AD6E060E656E7AEC45F079D053
:10BDF000380E04009EA8FDD7AD6E070E656E7AEC76
:10BE000045F06FD0390E04009EA8FDD7AD6E080E28
:10BE1000656E7AEC45F065D0410E04009EA8FDD712
:10BE2000AD6ED4EF47F05DD0420E04009EA8FDD762
:10BE3000AD6EA6EF4BF055D0430E04009EA8FDD783
:10BE4000AD6EE0EF4BF04DD0440E04009EA8FDD740
:10BE5000AD6E92EF4EF045D0450E04009EA8FDD782
:10BE6000AD6E4DEF4FF03DD0460E04009EA8FDD7BD
:10BE7000AD6E71EF55F035D0470E04009EA8FDD78A
:10BE8000AD6E27EF5AF02DD0480E04009EA8FDD7C6
:10BE9000AD6EDFD426D0490E04009EA8FDD7AD6E4E
:10BEA000010EEB6F83EC43F01CD04B0E04009EA8F8
:10BEB000FDD7AD6E487048B007D0CA0EF66E6B0E57
:10BEC000F76E5DEC36F006D0DE0EF66E6B0EF76E9A
:10BED0005DEC36F006D0000EF66E6C0EF76E5DEC83
:10BEE00036F046EC36F063C064F048B00BD01A0E62
:10BEF000F66E6C0EF76E5DEC36F004009EAAFDD770
:08BF0000AECF63F06ED6030022
:020000040030CA
:0E00000000C20E1E00858100000007A0070050
:00000001FF
